:100000000C94CB0B0C94050C0C94050C0C94050C67
:100010000C94050C0C94050C0C94050C0C94050C1C
:100020000C94050C0C94050C0C9478510C944852CB
:100030000C94104A0C94050C0C94050C0C94050CB3
:100040000C94050C0C94050C0C94050C0C94050CEC
:100050000C949D270C94874A0C94050C0C94050C69
:100060000C94050C0C94050C0C94050C0C94050CCC
:100070000C94050C0C94050C0C94050C0C94050CBC
:100080000C94050C0C94050C0C94050C0C94050CAC
:100090000C94050C0C94050C202020200053435296
:1000A000200020202020004341502000202020203C
:1000B000004E554D2000556E646566696E6564009E
:1000C00046756E6374696F6E0A00426173650A005B
:1000D0004C617965723A20004D306C6C790A0035BC
:1000E000001E001F00200021002200230024002504
:1000F00000260027002D002E002A00000053005487
:1001000000550056002B0014001A000800150017B7
:10011000001C0018000C00120013002F00300031EA
:100120000000005F0060006100000039000400165C
:1001300000070009000A000B000D000E000F00333D
:100140000034000000280000005C005D005E0057E5
:1001500000E10000001D001B000600190005001151
:10016000001000360037003800E50000000000599C
:10017000005A005B000000E000E300E20000000025
:10018000002C00000000000000E6000000E7002155
:1001900052E400000062000000630058000100010A
:1001A0000001000100010001000100010001000147
:1001B00000010001000100007C00000100010001BD
:1001C0000001000100010001000100010001000127
:1001D0000001000100010001000100010001000018
:1001E0000001000100010000000100010001000108
:1001F00000010001000100010001000100010001F7
:1002000000000001000000010001000100010001E8
:100210000000002078217823782478257826782714
:100220007828780578010001000000000001000135
:1002300000010000000100010001000000000001B9
:1002400000000000000000010000000100010001AA
:1002500000000001000000010001000A0025303309
:10026000326C62003A200025303258000A722F6347
:100270002030313233343536373839414243444502
:1002800046303132333435363738394142434445CC
:10029000460A001E0F0500047F3F1F6432146432BB
:1002A00014783C1E1E140A052223252628292A2CF0
:1002B0002D2F3032333536383A3B3D3E40424345B0
:1002C00047494A4C4E5051535557595A5C5E6062EB
:1002D000646668696B6D6F71737577797B7D7F81FB
:1002E000838587898A8C8E90929496989A9C9E9FFB
:1002F000A1A3A5A7A8AAACAEAFB1B3B4B6B8B9BB19
:10030000BCBEBFC1C2C3C5C6C7C9CACBCCCDCED087
:10031000D1D2D2D3D4D5D6D7D7D8D9D9DADADBDB74
:10032000DBDCDCDCDCDCDDDDDDDDDCDCDCDCDCDB0B
:10033000DBDBDADAD9D9D8D7D7D6D5D4D3D2D2D154
:10034000D0CECDCCCBCAC9C7C6C5C3C2C1BFBEBC47
:10035000BBB9B8B6B4B3B1AFAEACAAA8A7A5A3A1B8
:100360009F9E9C9A98969492908E8C8A898785837A
:10037000817F7D7B79777573716F6D6B696866645A
:1003800062605E5C5A5957555351504E4C4A49472A
:10039000454342403E3D3B3A3836353332302F2DCF
:1003A0002C2A292826252322FFAA7F554000000059
:1003B000000000000000000001010203040506081F
:1003C0000A0C0F1114181C2024292E33393F464CD7
:1003D000535B626A7179818A929AA2AAB2B9C1C842
:1003E000CFD5DCE1E7EBF0F4F7FAFCFDFEFFFEFD14
:1003F000FCFAF7F4F0EBE7E1DCD5CFC8C1B9B2AA5B
:10040000A29A928A8179716A625B534C463F393372
:100410002E2924201C1814110F0C0A0806050403A9
:1004200002010100000000000000000000000101C6
:1004300001010101010101020202020202020202A3
:100440000303030303030303040404040404040573
:100450000505050506060606060707070707080837
:100460000808090909090A0A0A0B0B0B0C0C0C0DE8
:100470000D0D0E0E0E0F0F0F101011111112121381
:10048000131414151516161717181819191A1A1BFC
:100490001B1C1D1D1E1E1F2020212222232424255B
:1004A0002626272829292A2B2C2D2D2E2F30313294
:1004B00032333435363738393A3B3C3D3E3F4041A4
:1004C00042434445464748494A4C4D4E4F5051538C
:1004D00054555658595A5B5D5E5F61626465666843
:1004E000696B6C6D6F7072737577787A7B7D7E80C7
:1004F00082838587888A8C8E8F91939596989A9C13
:100500009EA0A2A3A5A7A9ABADAFB1B3B5B7BABC26
:10051000BEC0C2C4C6C9CBCDCFD1D4D6D8DBDDDFF7
:10052000E2E4E7E9EBEEF0F3F5F8FAFDFFFD377AE8
:10053000585A000004E6D6B4460200210116000015
:1005400000742FE5A3E00814023A5D003D8889C6D7
:100550005436C3174FE4E293A3C96C75F133A3E596
:1005600088FCFA521D1694C22365D4CAEEA6F7720F
:100570000C7E8525E3F14272A52000808A827543B6
:10058000E31D42570F797C8EEBAB532F5345F04957
:100590003815D2A7FC8E7734C76D9186E90485A003
:1005A000F27760F3A5B20E81AD930C7D8A78764721
:1005B0000600CAE0BC18744345A6FD647BF6F472DD
:1005C0001DA3ADF88CB362424158405D61B718A0DD
:1005D000C8392F35DAF1E5871C65670B73C8BECFC4
:1005E000C64C9073103307730F8991D4769F9C4F3C
:1005F000949B5A2A0CA31A0F55449E990771869909
:100600002078FBCFCB3BBA352D55F9BBE1B22B5C43
:10061000666D7E49E1452A210286442B8A77B71E02
:10062000BE5F5D1303A6F49673724C007772D729F0
:10063000CD7D9454F9BBBC08B1881F1D8722E89476
:100640000234C006F44B74EA5662E960E3D83FB363
:10065000A345FC99FC498C0D68CC700B99B22953C9
:100660003677BF1131E51F58F03DBCC7ED0C20EACD
:100670004AB275148BD7F2A45F783254A2A0188CBA
:10068000DF91D47B269CCFA7C797407106C2F4F1B7
:10069000B45EC869BAA461576CD7BF8DE63623151E
:1006A000B92AE3BA797156FE43762C0BC3106EBD9E
:1006B0004902B48E344A4C8EE8DDC1B057177787B3
:1006C000A75F8891CA63A29DE2AC0FF3295D0E2655
:1006D0004FDEE4B68EEE2C391DF833F8B94F7E3676
:1006E000430B7F3EE1FC5557F91E698E9D8B862793
:1006F0005E6EF13DC27D30720FAEE215C968AFA1EA
:10070000DE7613BF93C79E2279788FD6B71E1F114E
:100710006922F1E1B8FE5682D48E55825BF9AA12A5
:100720009CDBCE5021E87DB2D71E0895CB9F3A02C4
:10073000B1D54330941A752BCC27BA395EC2DFFE8F
:10074000BD516D6473228B2C35F34FDDC2137F28AE
:10075000EDE34C0C76D95457DA97510081B1544CE3
:100760004E5F27716BE1BF7DFECF442669C8B5851A
:100770008121DD0D64ECF1E7B535F0052916ACF704
:10078000C00319B1C898000000935BC87F86756CE0
:10079000D40001D60495100000C93F0A64B1C467B3
:1007A000FB020000000004595A6F6C65645F6F66BD
:1007B0006620636D64206661696C65640A0000AE42
:1007C0006F6C65645F6F6E20636D64206661696C39
:1007D00065640A0000AF6F6C65645F72656E646586
:1007E0007239302064617461206661696C65640AE5
:1007F000006F6C65645F72656E646572206461741D
:1008000061206661696C65640A006F6C65645F7283
:10081000656E646572206F666673657420636F6DC4
:100820006D616E64206661696C65640A0064697359
:10083000706C61795F736574757032206661696C84
:1008400065640A0000DA0281FFD9F1DB20A4A62E3C
:10085000AF646973706C61795F666C6970706564B0
:10086000206661696C65640A0000A0C0D3006F6CEB
:1008700065645F696E697420636D64206E6F726D6C
:10088000616C20726F746174696F6E206661696C4F
:1008900065640A0000A1C8D3006F6C65645F696E6F
:1008A000697420636D64207365742031206661690A
:1008B0006C65640A0000AED580A81F408D1420002E
:1008C00007087F0807003E5B4F5B3E003E6B4F6BA7
:1008D0003E001C3E7C3E1C00183C7E3C18001C5711
:1008E0007D571C001C5E7F5E1C0000183C18000039
:1008F000FFE7C3E7FF00001824180000FFE7DBE76D
:10090000FF0030483A060E00262979292600407F4C
:1009100005050700407F05253F005A3CE73C5A008B
:100920007F3E1C1C0800081C1C3E7F0014227F22F6
:1009300014005F5F005F5F0006097F017F000066B3
:1009400089956A0060606060600094A2FFA29400D4
:1009500008047E04080010207E20100008082A1CCD
:100960000800081C2A0808001E10101010000C1E99
:100970000C1E0C0030383E383000060E3E0E0600CD
:1009800000000000000000005F00000000070007FA
:100990000000147F147F1400242A7F2A12002313DE
:1009A0000864620036495620500000080703000022
:1009B000001C224100000041221C00002A1C7F1C58
:1009C0002A0008083E08080000807030000008086F
:1009D0000808080000006060000020100804020001
:1009E0003E5149453E0000427F400000724949495E
:1009F00046002141494D33001814127F100027454D
:100A0000454539003C4A4949310041211109070057
:100A1000364949493600464949291E00000014005C
:100A200000000040340000000008142241001414AB
:100A30001414140000412214080002015909060090
:100A40003E415D594E007C1211127C007F4949499C
:100A500036003E41414122007F4141413E007F49F5
:100A6000494941007F09090901003E414151730094
:100A70007F0808087F0000417F4100002040413F7F
:100A800001007F08142241007F40404040007F0267
:100A90001C027F007F0408107F003E4141413E0060
:100AA0007F09090906003E4151215E007F0919298D
:100AB000460026494949320003017F0103003F40B7
:100AC00040403F001F2040201F003F4038403F0073
:100AD0006314081463000304780403006159494D4A
:100AE0004300007F41414100020408102000004102
:100AF00041417F00040201020400404040404000A8
:100B00000003070800002054547840007F28444424
:100B10003800384444442800384444287F0038547E
:100B20005454180000087E09020018A4A49C780000
:100B30007F080404780000447D4000002040403DD0
:100B400000007F102844000000417F4000007C042A
:100B5000780478007C080404780038444444380061
:100B6000FC182424180018242418FC007C08040411
:100B7000080048545454240004043F4424003C40DA
:100B800040207C001C2040201C003C4030403C00A9
:100B90004428102844004C9090907C004464544CAD
:100BA00044000008364100000000770000000041CA
:100BB000360800000201020402003C2623263C0005
:100BC000000000000000404040F0F8F8FF38FFF857
:100BD000F83FF8F8FF38FFF8F8F040404000000018
:100BE00000000080C0C0C0800000C0C080000000C5
:100BF00080C0C000C0C0000080C0C0000000000075
:100C0000C0C0C0C0C000C0C00000000000000000A4
:100C100000000000000000000000000000000000D4
:100C200000000000000000000000000000000000C4
:100C3000000000000000000000000000000000C0F4
:100C4000F0F8FC3E1E06010000007F4141417F009C
:100C50007F4141417F000080C0E07E5B4F5BFEC072
:100C60000000C000DCD7DEDEDED7DC00C000000004
:100C70000000000000000000000000000000000074
:100C8000000000000000494949FFFFFFFFE0DFBF0F
:100C9000BF00BFBFDFE0FFFFFFFF49494900000081
:100CA00000001F3F6060E0BF1F007F7F071E381EEF
:100CB000077F7F007F7F0E1F3B71600000000000F8
:100CC0007F7F0C0C0C007E7E007F7E0303007F7E06
:100CD00003037E7E03037F7E000F3E703C063C7064
:100CE0003E0F00327B49493F7E007F7E0303001E9A
:100CF0003F69696F2600000000000000000000034B
:100D00000F1F3F3C7870600000007F4141417F0031
:100D10007F4141417F00307B7F7830202030787FD9
:100D20003B0003000F7F0F0F0F7F0F000300000039
:100D300000000000000000000000000000000000B3
:100D4000000000000000010101070F0F7F0F7F0F5F
:100D50000F7E0F0F7F0F7F0F0F07010101000000B3
:100D60000000000000000001010000000000000081
:100D70000000000000000000000000000000000073
:100D80000000000000000000000000000000000063
:100D90000000000000000000000000000000000053
:100DA0000000000000000000000000000000000043
:100DB0000000000000000000000000000000000033
:100DC0000000000000000000000000000000000023
:100DD0000000000000000000000000000000000013
:100DE0000000000000000000000000000000000003
:100DF00000000000000000000000000000000000F3
:100E0000313A0964656C6179282A31306D73293A69
:100E10002025750A323A09696E74657276616C280C
:100E20006D73293A2025750A333A096D61785F732D
:100E3000706565643A2025750A343A0974696D65F0
:100E40005F746F5F6D61783A2025750A353A0977CE
:100E50006865656C5F6D61785F73706565643A2085
:100E600025750A363A09776865656C5F74696D6542
:100E70005F746F5F6D61783A2025750A00703A09DA
:100E80007072696E742076616C7565730A643A09D4
:100E90007365742064656661756C74730A75703A65
:100EA000092B310A646E3A092D310A6C743A092B08
:100EB00031300A72743A092D31300A4553432F718B
:100EC0003A09717569740A0A7370656564203D207A
:100ED00064656C7461202A206D61785F737065654C
:100EE00064202A2028726570656174202F2074693F
:100EF0006D655F746F5F6D6178290A7768657265EB
:100F00002064656C74613A20637572736F723D255D
:100F1000642C20776865656C3D25640A53656520FF
:100F2000687474703A2F2F656E2E77696B697065DF
:100F30006469612E6F72672F77696B692F4D6F75CA
:100F400073655F6B6579730A004D3E20004D257512
:100F50003A25733E20003F0A003D2025750A003FD8
:100F60000A0064656661756C74730A0025750A0071
:100F70003F0A000A092D2056616C756573202D0A01
:100F800000710A000A092D204D6F7573656B657934
:100F9000202D0A003F00433E20004C25640A000A31
:100FA000092D20537461747573202D0A686F737452
:100FB0005F6B6579626F6172645F6C656473282929
:100FC0003A20253032580A6B6579626F6172645F2E
:100FD00070726F746F636F6C3A20253032580A6BF1
:100FE0006579626F6172645F69646C653A2025306F
:100FF00032580A6B65796D61705F636F6E66696701
:101000002E6E6B726F3A20253032580A74696D6506
:10101000725F72656164333228293A202530386C5A
:10102000580A002573000A092D20436F6E736F6CF8
:1010300065202D0A4553432F713A09717569740A69
:101040006D3A096D6F7573656B65790A000A092D34
:10105000204D61676963202D0A443A094465627531
:1010600067204D65737361676520546F67676C65B2
:101070000A583A094D61747269782044656275674F
:10108000204D6F646520546F67676C65202D205379
:10109000686F77206B65797072657373657320690B
:1010A0006E206D617472697820677269640A4B3AC8
:1010B000094B6579626F61726420446562756720CF
:1010C000546F67676C65202D2053686F77206B65C0
:1010D000797072657373207265706F72740A4D3A1D
:1010E000094465627567204D6F75736520546F679D
:1010F000676C650A563A0956657273696F6E0A53D2
:101100003A095374617475730A433A094163746907
:101110007661746520436F6E736F6C65204D6F64EC
:10112000650A46312D4631303A0953776974636850
:1011300020746F204C6179657220302D392028464B
:101140003130203D204C30290A302D393A0953776F
:101150006974636820746F204C6179657220302D4A
:10116000390A47524156453A0953776974636820F2
:10117000746F204C6179657220302028616C746531
:10118000726E617465290A423A094A756D7020745D
:101190006F20426F6F746C6F616465720A455343D0
:1011A0003A094A756D7020746F20426F6F746C6FCE
:1011B000616465722028616C7465726E6174652962
:1011C0000A453A095072696E7420454550524F4D98
:1011D0002053657474696E67730A4241434B5350E0
:1011E0004143453A09436C65617220454550524F71
:1011F0004D0A4E3A094E4B524F20546F67676C654B
:101200000A006261636B6C696768745F636F6E6626
:1012100069672E7261773A20253032580A2E656E42
:1012200061626C653A2025750A2E6C6576656C3AAC
:101230002025750A006B65796D61705F636F6E665E
:1012400069672E7261773A20253032580A2E7377FB
:1012500061705F636F6E74726F6C5F636170736CEB
:101260006F636B3A2025750A2E636170736C6F6330
:101270006B5F746F5F636F6E74726F6C3A2025756D
:101280000A2E737761705F6C63746C5F6C6775694D
:101290003A2025750A2E737761705F7263746C5FF4
:1012A000726775693A2025750A2E737761705F6CD5
:1012B000616C745F6C6775693A2025750A2E7377C7
:1012C00061705F72616C745F726775693A20257531
:1012D0000A2E6E6F5F6775693A2025750A2E73773F
:1012E00061705F67726176655F6573633A2025752B
:1012F0000A2E737761705F6261636B736C617368F0
:101300005F6261636B73706163653A2025750A2EB5
:101310006E6B726F3A2025750A2E737761705F6568
:1013200073636170655F636170736C6F636B3A20A8
:1013300025750A0064656275675F636F6E6669672D
:101340002E7261773A20253032580A2E656E61621E
:101350006C653A2025750A2E6D61747269783A20A1
:1013600025750A2E6B6579626F6172643A20257566
:101370000A2E6D6F7573653A2025750A00656563E1
:101380006F6E6669673A0A64656661756C745F6C56
:10139000617965723A20256C750A003F004E4B5208
:1013A0004F3A206F66660A004E4B524F3A206F6EDE
:1013B0000A000A6D6F7573653A206F66660A000A47
:1013C0006D6F7573653A206F6E0A000A6B657962FE
:1013D0006F6172643A206F66660A000A6B65796213
:1013E0006F6172643A206F6E0A000A6D61747269EF
:1013F000783A206F66660A000A6D61747269783AFD
:10140000206F6E0A000A64656275673A206F66662F
:101410000A000A64656275673A206F6E0A000A0A5C
:101420004A756D70696E6720746F20626F6F746C9F
:101430006F616465722E2E2E2000433E2000436CA7
:10144000656172696E6720454550524F4D0A00290B
:101450000A002575002F002575005D280025640011
:101460002000256400200025640020002564007C05
:101470000025303258006D6F7573656B6579205BA0
:1014800062746E7C782079207620685D28726570A1
:101490002F61636C293A205B00504F52514A4D4BEB
:1014A0004E2A4C2F30B6B7ABACBBBCA9AABDBECF41
:1014B000D0CDCEDBDCD9DA0D0E0B0F1A05080509ED
:1014C00005071811130408120C00000000000000AA
:1014D000002A2B280000000000000000000000008F
:1014E0000000000029000000002C1E3420212224CE
:1014F000342627252E362D3738271E1F202122235C
:101500002425263333362E37381F040506070809ED
:101510000A0B0C0D0E0F10111213141516171819B3
:101520001A1B1C1D2F3130232D3504050607080911
:101530000A0B0C0D0E0F1011121314151617181993
:101540001A1B1C1D2F3130354C000000000000001C
:10155000000000000000000000000000000000008B
:10156000000000000000000000000000007E0F00EE
:10157000D4FFFFFFC7000000785B575D005B535D41
:10158000005B525D005B445D005B435D001C0376C5
:1015900000690061006C003A0066003600340063A8
:1015A00000320062003300630000000C034D003085
:1015B000006C006C00790000002003540068006596
:1015C0000020004B0065007900200043006F006D93
:1015D00000700061006E0079000000040309040936
:1015E000027400040100A0FA0904000001030101D3
:1015F00000092111010001224400070581030800B0
:101600000109040100020300000009211101000189
:1016100022220007058203200001070503032000A2
:101620000109040200010300000009211101000169
:1016300022B600070584032000010904030001030A
:101640000000000921110100012215000705850392
:1016500020000112010002000000084B54040001A8
:1016600000010203010631FF0974A101097515008B
:1016700026FF00952075088102C00660FF0961A160
:10168000010962150026FF00952075088102096393
:10169000150026FF00952075089102C0050109027A
:1016A000A10185020901A1000509190129081500F8
:1016B000250195087501810205010930093115815F
:1016C000257F95027508810609381581257F9501CA
:1016D00075088106050C0A38021581257F9501756C
:1016E000088106C0C005010980A101850319012AEE
:1016F000B700150126B700950175108100C0050CD3
:101700000901A101850419012AA002150126A002E0
:10171000950175108100C005010906A10185060526
:101720000719E029E71500250195087501810205D3
:1017300007190029EF1500250195F07501810205B3
:101740000819012905950575019102950175039107
:1017500001C005010906A101050719E029E71500E7
:10176000250195087501810295017508810105071C
:10177000190029FF150026FF009506750881000550
:101780000819012905150025019505750191029596
:101790000175039101C011241FBECFEFD0E2DEBF5F
:1017A000CDBF04B603FE18C08091DD0D9091DE0D13
:1017B000A091DF0DB091E00D8730904BA740B04B6A
:1017C00059F41092DD0D1092DE0D1092DF0D109283
:1017D000E00DE0E0F0EF099513E0A0E0B1E0EAED04
:1017E000FDEA00E00BBF02C007900D92AE34B107D6
:1017F000D9F72DE0AEE4B3E001C01D92AD3DB207D4
:10180000E1F70E94301F0C941E560C940000FF93C9
:10181000EF93E0914E03F0914F03309709F0099553
:10182000EF91FF910895FC018591803011F0EFDF79
:10183000FBCF0895FF27E0E230E247FF0CC041955F
:1018400097FF09C0EDE26095709580959095611DB8
:10185000711D811D911D27FF02C0219530E350E2CB
:10186000AA27660F771F881F991FAA1FA41710F0B9
:10187000A41B63955A95A9F7AA3008F0A95FA05D4B
:10188000AF93F395611571058105910541F7ED322F
:1018900011F4EF93F395F21718F43F93F395FBCF00
:1018A0008F91B5DFFA95E1F70895E991F991859166
:1018B000803021F0853219F0AADFF9CF089520E0B9
:1018C000E89455915532C1F3503311F46894559111
:1018D0005A3348F4505390F3220F022E220F220F56
:1018E000200D250FF4CF0EF421958991999153364F
:1018F00019F3533729F1533559F1BC01882799273A
:10190000E8945C3621F48991999168945591543604
:1019100039F446EF7EF077FF0DC08FEF9FEF0AC0DE
:1019200055374AE039F0583540E121F0523642E06F
:1019300009F00895FF93EF937DDFEF91FF91B7CF0B
:10194000FF93EF93FC0181918030B9F360DFFBCF0F
:10195000FF93EF9368DFF1CFDF93CF93CDB7DEB77F
:101960002596A3DFCF91DF9108955098589A51980A
:10197000599A279A2F9A0C947D19CF9360E088ED9D
:1019800090E00E94702E60E080ED90E00E94702E4A
:1019900080917A0333D2811541F0813061F160E0AA
:1019A00086EB90E00E94812E05C060E08AEC90E01A
:1019B0000E94702E0E94D547C82F81EB90E0C0FD99
:1019C00002C08CEA90E060E00E94702E87EA90E00E
:1019D000C1FD02C082EA90E060E00E94702E8DE9B5
:1019E00090E0C2FD02C088E990E060E00E94702EA5
:1019F00080E0CF91089560E080EC90E0D9CF823014
:101A0000D0F46530C0F44331B0F4E42FF0E093E15A
:101A1000699FE00DF11D112490E091958195910948
:101A20008F759927E80FF91FEE0FFF1FE152FF4F47
:101A300085919591089581E090E008959C019A9593
:101A400081159F4118F5F32FF270EE27832F8170D7
:101A5000732F74706627532F5870442734FF0CC0BF
:101A60008295807FEF2B09F08062672B09F08064FC
:101A7000452B69F080680895EF2B09F08260672B91
:101A800009F08460452B19F08860089580E008957E
:101A9000CF93DF93EB01D2DFFE010995DF91CF9168
:101AA0000895CF93DF93EC01805E9109089720F0B1
:101AB0006AEF72E1209711F461EE70E1CE01E8DF88
:101AC0008C2F7DD2DF91CF910895CF93DF93EC01DE
:101AD00006D3CE01805E9109089720F06FEF72E186
:101AE000209711F466EE70E1CE01D2DFDF91CF9145
:101AF000089581E0089581E00895FBCF089581E085
:101B0000089581E0089581E00895FDCF0895089536
:101B10000895FDCF089508950895A6E0B0E0E3E9A3
:101B2000FDE00C94B05449835A839E833091550351
:101B300089819A81311117C03E81311589F02115B3
:101B400079F090D6182F682F89819A816AD6698199
:101B50007A81812F0E94781B2696E3E00C94CC5466
:101B600071D6182FF4CF7ED669817A81F3CFFC012C
:101B7000262F87819085009739F4408151816281B9
:101B8000738184819581C9CF0895CF93DF93D82F36
:101B9000C92F61E0ECDF6D2F7C2FADDF811106C016
:101BA00080E090E08170DF91CF91089561E08D2F0A
:101BB0009C2FDDDF6D2F7C2FA0DF811589F361E085
:101BC0008D2F9C2FD4DF6D2F7C2F0E945333EACFB3
:101BD0000F931F93CF93DF93D82FC92F60E0C7DFF8
:101BE0008C016D2F7C2F94DF6D2F7C2FC80191DF2E
:101BF000DF91CF911F910F91089591E001C0990F4E
:101C00008A95EAF7892F66C5CF93C82F81E00C2EFD
:101C100001C0880F0A94EAF70E9437198C2FEDDF74
:101C2000CF91089581E0089581E00895FBCF089554
:101C3000CF93C82FFAD48C2FF7DF8C2FF7DF2FEF3D
:101C400084E39CE0215080409040E1F700C0000018
:101C5000CF91089581E0ECDF0C94AB4A80E0E8DF9F
:101C60000C94CF4A0F931F93CF93DF93EC018B011A
:101C70000E94C444811521F061E0C80178DFEC01C5
:101C8000F801858181110E94CA25B801CE010E9408
:101C90001E41811509F484C0B801CE010E9478412B
:101CA000811509F47DC0B801CE012BDF811509F43F
:101CB00077C0B801CE0129DF811509F471C0B801E0
:101CC000CE010E941246811509F46AC0B801CE0106
:101CD0000E943E2C811509F463C0B801CE010E9418
:101CE000CA26811509F45CC0B801CE010E948D306E
:101CF000811509F455C0B801CE010E94E94481154F
:101D000009F44EC0B801CE010E944544811509F482
:101D100047C0B801CE010E94553D811509F440C06D
:101D2000B801CE010E947A3C8115D1F1B801CE01F3
:101D30000E944A1F8115A1F1B801CE010E94804581
:101D4000811571F1B801CE010E94871C811541F106
:101D5000B801CE010E94A53C811511F1F8018581E1
:101D6000811581F0CA35FCE7DF0721F170F4C1303D
:101D7000ECE7DE07E9F0C330FCE7DF07B9F0C11597
:101D8000DC4769F0C801BBDE0CC0CB35ECE7DE07F1
:101D9000A1F0CC35DC47B1F70E94F418F3CF5ADF3D
:101DA00080E0DF91CF911F910F9108950E942C192F
:101DB00055DFF6CF0E94FB18E5CF0E94FD18E2CF59
:101DC000CF93DF93D82FC92F61E0D1DE6D2F7C2F09
:101DD00049DFDF91CF9108959EDE0E94E54980E0C2
:101DE0000E94AD267DD00C94AD2F0E9406267AD09D
:101DF00093DE0C94E9490C9465540895982F9295BC
:101E00009F7024E0911102C020E0982F892F8695C1
:101E10008695811511F02E5F982F892F8695820F58
:101E200008958295982F990F990F9C7C8695869599
:101E30008373982B892F880F8A7A96959575892BAD
:101E40000895CF93DF93D92FECDFC82F8D2FE9DFD3
:101E50009C2FDF91CF9108950F931F93CF93DF9322
:101E60008C01CB01EEDFEC01C801EBDF8C01BE0180
:101E700080E090E0CB017727662720E030E0602B00
:101E8000712B822B932BDF91CF911F910F9108958E
:101E900081E0089580FF08C05A9A81FF07C05B9ACD
:101EA00082FF06C05C9A08955A98F7CF5B98F8CFE6
:101EB0005C980895CF93DF93D82FEADFC82F811560
:101EC00011F08D2FE7DF8C2FDF91CF910895529A7B
:101ED0005A98539A5B98549A5C980895EBCF08955A
:101EE00080E0FCCF0E94C647F9CFCF930E94C6473F
:101EF000C82F809150038C1771F0C09350030E943B
:101F00007B4A6093510370935203809353039093E1
:101F100054038C2FE3DFCF910895AFE0B0E0E3E905
:101F2000FFE00C94AF544A875B876C877D878E8770
:101F30009F8791110E94E1171F821886198626E05B
:101F4000FE013A96CE010196DC0101900D922A9590
:101F5000E1F72091F8098C0122FF0AC0EED7811524
:101F600019F082E00E94CD18CED781110E9434185A
:101F70008D8181110EC009811A812B813C814D8197
:101F80005E816F81788589853BD72F96E4E00C943C
:101F9000CB54C801FADD8111EECFF7CFFC0184816B
:101FA000813019F48081918185C40895611521F0F3
:101FB0000E94B73E0C94703F0E94F83EFBCFCF9337
:101FC000C82F8115C9F08238C9F40E94D54781FD18
:101FD00013C089E30E9416490E949E182FEF37EE26
:101FE00083E0215030408040E1F700C0000089E3E9
:101FF0000E942D490E949E18CF9108958338A1F424
:102000000E94D54780FDF8CF83E50E9416490E94C3
:102010009E189FEF21EE34E0915020403040E1F7D0
:1020200000C0000083E5E4CF8438A1F40E94D547C6
:1020300082FDE2CF87E40E9416490E949E188FEF2E
:1020400091EE24E0815090402040E1F700C0000074
:1020500087E4CECF8CEF8C0F813A98F48C2F0E94BE
:1020600007388111C9CF8C2F0E948848811529F02B
:102070008C2F0E942D490E949E188C2F0E94164979
:10208000B9CF80E28C0F883040F4C77081E001C086
:10209000880FCA95EAF770D7ADCF8BE58C0F8330E8
:1020A00038F42C2F2452330BC9010E940A48A4CFC4
:1020B000E8E5EC0FEB3150F4F0E0EE0FFF1FE05CD1
:1020C000FE4F808191810E94324896CF83E38C0F2E
:1020D000833108F091CF61E08C2F68DF8DCF8115BF
:1020E00009F451C0823871F40E94D54781FF4BC07A
:1020F00089E30E9416490E949E1889E30E942D4997
:102100000C949E18833859F40E94D54780FF3BC039
:1021100083E50E9416490E949E1883E5EFCF84381C
:1021200059F40E94D54782FF2EC087E40E941649C9
:102130000E949E1887E4E2CF9CEF980F913AF0F24C
:1021400090E2980F983048F4877091E001C0990FA1
:102150008A95EAF7892F16D7D3CF9BE5980F93304E
:1021600020F480E090E00C940A4898E5980F9B31A9
:1021700020F480E090E00C94324893E3980F933180
:1021800010F460E013CF08951F93CF93DF93182FBF
:10219000EB0115DF209731F4812FA1DFDF91CF9183
:1021A0001F9108958FE99FE00197F1F700C00000AB
:1021B0002197F0CF60E570E0893311F060E070E0C6
:1021C000E3CF811511F0D8D6B9C70895811511F064
:1021D000D9D6B4C70895A0E0B0E0E1EFF0E10C94E7
:1021E000AB546C01D62FC72FFC010581F6801F2D43
:1021F00012951F70B6D6E82E8115E9F0E02E011574
:10220000D1F08C2F807F803461F080E28D0F883098
:10221000E0F08C2F807E803221F4D230B0F01115A6
:10222000A1F08091F80982FF10C082E0B6D799D65C
:1022300091E0E82EE926EC2FE295EF70C03C78F5AE
:10224000F0E0E05EF94A0C945C54E12CF4CF1C2FD2
:102250001F70C03110F01295107F011581F011151B
:1022600049F080E28D0F883010F0D11105C0812F28
:1022700083D664D78D2F42C0812F92D6FACF8D2F6F
:102280002EDF111561F080E28D0F883010F0D11132
:1022900003C0812F77D602C0812F88D64FD7E11493
:1022A00009F4C5C046D680FDC2C0F60115823BD6F2
:1022B00033D2C60181D137D639D2B9C0FC2FFF70D5
:1022C000FF2EC07FC03219F0F29480EFF822D115B2
:1022D00049F0D13009F442C0011509F44BC0111581
:1022E000C9F0C8CF8091F80982FD10C0011541F0F6
:1022F000F11419F08F2D40D621D780E060DECFCFCA
:1023000080E0EDDEF11459F28F2DC4CF0115A1F05C
:10231000111103C08F2D55DFC2CF113019F48F2D4D
:1023200074D6BDCF153009F0BACF8F2D4ADF8F2D6F
:1023300082D68F2D4FD6B3CF111107C08F2D46DF18
:102340008F2D79D68F2D52D6AACF113009F0A7CF75
:1023500010D68F21811509F4A2CFF0CF011521F0FD
:10236000163008F09CCFD6CF153008F098CF8F2DBF
:102370002DDF95CF1115D9F3D93349F42FEF87EE1F
:1023800093E0215080409040E1F700C000008D2F85
:10239000A6DE85CF8C2F869586958370811569F092
:1023A000813009F07CCF8D2F9C2F9370011102C0DA
:1023B00080E090E00E94324872CF8D2F9C2F937066
:1023C000011102C080E090E00E940A4868CF602FAF
:1023D0008D2FECDD64CF8C2F8370811133C0011100
:1023E00023C04D2F429546954770440F440F8D2FC3
:1023F0008F70042E01C0880F0A94EAF72D2F2071E8
:10240000D4FF07C02FE030E001C0220F4A95EAF761
:102410002095C695C695C370822BC23079F0C33023
:1024200079F0C13049F05CD10E94C64757DDCDB785
:10243000DEB7E8E00C94C7544FD1F6CF55D1F4CFB6
:1024400049D1F2CF011531F1C0FFEECF4D2F4295AA
:1024500046954770440F440F8D2F8F70042E01C096
:10246000880F0A94EAF72D2F2071D4FF07C02FE0C0
:1024700030E001C0220F4A95EAF72095C695C6952F
:10248000C370822BC23059F0C33059F0C13029F0EB
:1024900069D1CACF823040F2D9CF60D1C5CF66D1E1
:1024A000C3CF2CD1C1CFCF70011529F08C2F34D1DF
:1024B0008D2F87DEB9CF8D2F89DE8C2F37D1B4CF0A
:1024C000D23F31F168F4D03FC1F0D13F89F001151E
:1024D00009F448C0111509F442C08D2F70DDA4CF56
:1024E000D33FE1F0D43F99F78091F80982FD1EC0F7
:1024F0008C2F8F71011511F30FC0011539F01530B4
:1025000008F092CF8C2F8F711FD18ECF1630F8CF5D
:102510008C2F8F710111D2CFFFD086CF011521F002
:102520008C2F8F71F2D080CFEED07ECF011579F055
:1025300000D5843021F429D68C2F8F71BFCF63E072
:10254000153008F071CF8C2F8F7105D66DCF1530F7
:1025500018F01BD664E0F7CF81E01FD665CF8C2F33
:102560008F71DACF111541F3D93349F4EFEFF7EE5C
:1025700023E0E150F0402040E1F700C000008D2F43
:10258000AEDD52CF0F931F93CF93DF93EC018F817A
:102590009885009761F09FD78C01ECD09AD0B80154
:1025A000CE0119DEDF91CF911F910F9108956881BF
:1025B00079818D818AD1F0CFCF93DF93EC018C812B
:1025C000811581F0CE01FCDB81110FC0CAD48115C9
:1025D00049F08D81811531F08091F80982FF02C0A8
:1025E00082E0DBD5DF91CF910895CE01CBDFCE0124
:1025F000EFDAF8CF811511F0D3D4A0C50895811575
:1026000011F0D4D49BC5089580E090E00E940A4860
:1026100080E090E00E943248D4D490D50E942540BA
:102620000C94703F0E944449EFCFB4D4FBCF282FC5
:1026300092959F70963099F060F4925F9F709230FF
:1026400030F4203FB1F038F481E0283E38F080E0EB
:1026500008959A5FF3CF81E0243FC9F7089591E090
:10266000813F09F090E081E0283E08F080E0892B6E
:10267000089581E00895FC018481811551F08781DE
:102680009085009711F027D7D2CF8081918112D108
:10269000FBCF80E00895A6E0B0E0E1E5F3E10C9423
:1026A000B1542696E2E00C94CD54A9E0B0E0EBE5FD
:1026B000F3E10C94AF542996E4E00C94CB540895C4
:1026C000FECF0895FDCF0895FADFFCDF80937B03F2
:1026D00008950895F9CF089590917B03892BF4CF45
:1026E00090917B038923F0CF90917B038927ECCFD6
:1026F000E6CF0895FDCF0895E2CF0895FDDFFADF1C
:1027000080937A03089580E0F9CF91E001C0990F9A
:102710008A95EAF7892FF2CF21E030E001C0220F3D
:102720008A95EAF780917A03822BE8CF21E030E0A6
:10273000A90102C0440F551F8A95E2F7CA0180958E
:1027400090917A038923DACF21E030E001C0220F93
:102750008A95EAF780917A038227D0CF90917A0305
:10276000892BCCCF90917A038923C8CF90917A039B
:102770008927C4CF08959B01677091E001C0990F2C
:102780006A95EAF763E0369527956A95E1F7B9010E
:10279000660F771F260F371FFA01E20FF31F40E085
:1027A00050E0682F70E08191DF019B01042E02C090
:1027B000369527950A94E2F7217021952827292339
:1027C00028272E934F5F5F4F4330510561F70895DF
:1027D0009C01A82FA77083E0369527958A95E1F78D
:1027E000C901880F991F820F931FFB01E80FF91F82
:1027F00040E050E080E0219130E00A2E02C03695A2
:1028000027950A94E2F721703327042E01C0220F86
:102810000A94EAF7822B4F5F5F4F4330510559F717
:102820000895282F862F953060F4233150F4622FBD
:1028300070E023E1929F600D711D112446E553E085
:102840009ACF0895292F953058F4833148F490E0B9
:1028500066E573E033E1239F800D911D1124B8CF0D
:1028600080E00895A0E0B0E0E8E3F4E10C94AC541B
:102870007C0100917A0380917B03082BC3E0D0E0B8
:1028800010E0C8010C2E02C0959587950A94E2F7D6
:1028900080FD09C02197A8F7D12C8D2DCDB7DEB7CB
:1028A000E7E00C94C854DC2EB7018C2F3BD701977E
:1028B00089F3F3CFCF93DF93D82FC92FD3DF6D2FB9
:1028C0007C2F30D7DF91CF9108951F93CF93DF9363
:1028D000162FD72F90915503911539F0862F972FEA
:1028E000E9DFDF91CF911F910895811569F0862F5F
:1028F000972FB8DFC82F682F812F9D2F92DF612F70
:102900007D2F8C2F0FD7EDCF862F972F9BDFC82FD2
:10291000F6CFE1E0F0E0DF0102C0AA0FBB1F6A952D
:10292000E2F7BD01DF0102C0AA0FBB1F4A95E2F723
:102930006A2B01C0EE0F2A95EAF7962F982396137B
:1029400002C08E2B0895E0958E230895242F462FE4
:10295000682F80917A03DDDFD1CEEF92FF920F9343
:102960001F93CF93E0917C03C9E080917D038E1388
:1029700006C0CF911F910F91FF90EF900895EE2E1A
:10298000F12CCE9FF0011124E258FC4F00811181FF
:10299000228133814481558166817781808585DEFE
:1029A000F7013196E770E1CF0F931F930091C603B3
:1029B0001091C7032091C8033091C9034091CA0305
:1029C0005091CB036091CC037091CD038091CE03E5
:1029D0006CDE1F910F910895E0917C0390917D032F
:1029E00029E0E91302C080E00895AE2FB0E02E9FE9
:1029F000F0011124E258FC4F3181361306C03081BA
:102A0000381303C03581341304C0FD013196E770DB
:102A1000E8CF81E00895A0E0B0E0E1E1F5E10C94B9
:102A2000AC548091CC03803108F048C08091CB0336
:102A3000811509F443C0C0917C0389E0D82E8091B0
:102A40007D038C17D9F1EC2EF12CDC9EE0011124D2
:102A5000FE01E258FC4F84818115A9F1918180919A
:102A6000C703981330C090818091C60398132BC080
:102A70008581811128C0028113818091C8039091C2
:102A8000C903081B190B60E086EC93E070D866EC74
:102A900073E00E94112C08171907A8F48091CC0349
:102AA0008F7080618093CC03CC57DC4F88818F700E
:102AB0008061888386EC93E07FDD4FDFCDB7DEB7A2
:102AC000E7E00C94C854E7012196C770B8CFAFE097
:102AD000B0E0EDE6F5E10C94A4548C0186E0F80139
:102AE000DE011A9601900D928A95E1F7F801F580C2
:102AF000748086ECA82E83E0B82E8091CA038111E1
:102B000017C0711409F419C1F11409F46EC1C80198
:102B1000B2DD811509F469C189E0F801D5010190A0
:102B20000D928A95E1F7C50139DA75DF3DDF05C100
:102B3000C280D380E090CB038091C8039091C903F9
:102B40004601881A990AE11409F4FAC0608051809C
:102B500060E086EC93E00BD866EC73E00E94112CE9
:102B60008816990608F0B3C0711409F4E6C0909174
:102B7000C703F80121818091CC03803108F05EC049
:102B8000291322C02091C603908129131DC04091B2
:102B9000CD035091CE032781308542175307A1F40E
:102BA000F11046C08F7080618093CC03FDDE86EC0F
:102BB00093E002DD8091CC03F8018683F12C8F2D08
:102BC0002F96EFE00C94C054F11032C040E0652D18
:102BD000862D02DF40E0652D862DFEDEF82E811168
:102BE000EDCF8A859B8566DE292F22952F70903444
:102BF00050F49F70223078F0911589F0F801968199
:102C0000903168F4DCCF2A5F2F70223060F0C80169
:102C1000D3DCFE2CD4CF911511F0811581F2805EAA
:102C2000883068F2F4CF803F50F2815F8330F9CF73
:102C30008091CC0381608093CC03C0CF29131CC04A
:102C40002091C6039081291317C04091CD03509164
:102C5000CE03278130854217530771F4F1100CC061
:102C60008683C801A9DC89E0F801A6ECB3E00190F5
:102C70000D928A95E1F75ACFC801FDDC811509F460
:102C8000B4C0F11409F4B1C08091CC038032B0F02B
:102C90002091C6033091C7033A832983DC82CB821B
:102CA0009091CA039D831E828F838091CD03909162
:102CB000CE0399878887CE0101967EDC89E0F801F2
:102CC000A6ECB3E001900D928A95E1F72ECF8091AA
:102CD000CC03803188F44A855B856C857D858E8543
:102CE0009F85D9DC86EC93E067DC89E0F5011192E1
:102CF0008A95E9F759DE62CF7114F9F02091C70384
:102D0000F80191812913B8CF2091C603908129132E
:102D1000B3CF4091CD035091CE0327813085421728
:102D2000530709F0A9CFF110A7CF8683C80144DC6F
:102D300089E0F50111928A95E9F7FF24F3943FCFDA
:102D400060E086EC93E00E94B70D66EC73E00E94B1
:102D5000112C8816990608F04BC0711471F3F11408
:102D600009F443C09091C703F8018181981334C0DE
:102D70009091C603808198132FC02091CD0330918C
:102D8000CE03878190852817390731F58091C803D4
:102D90009091C903C81AD90AF8ECCF16D10498F457
:102DA0008091CC0380FD0FC0803168F0F8018683EC
:102DB000982F907F903F09F454CF982F907F905F89
:102DC0008F70892B4DCF89E0F801A6ECB3E001901C
:102DD0000D928A95E1F7B1CFC8014DDC81116ECF1C
:102DE0008091CC0381608093CC03C801E5DBA5CF43
:102DF0004A855B856C857D858E859F854CDC75CF8E
:102E0000A2E1B0E0E6E0F7E10C94AE540A871B873C
:102E10002C873D874E875F87688B798B8A8BCE01A5
:102E20000A9655DE4E858115B9F0411549F00A859F
:102E30001B852C853D855F85688979898A8935DC84
:102E400089E0F82E80917C0390917D03891338C02E
:102E50006296E5E00C94CA5489E0FE013A96DE01E0
:102E6000119601900D928A95E1F7411549F3A091D1
:102E70007D038A2F90E001968770992720917C032B
:102E80002817190681F099E09A9FD0011124A258C1
:102E9000BC4FFE01319601900D929A95E1F7809317
:102EA0007D035BDDCDCFC1DB10927D0310927C03EF
:102EB00089E0E6ECF3E0DF011D928A95E9F7C0CFE7
:102EC000F89EC001112482589C4F01DE811509F43F
:102ED000BFCFE0917C03FE9EF0011124E258FC4F2D
:102EE00000811181228133814481558166817781FE
:102EF0008085DBDB80917C0390E0019687709927C9
:102F000080937C039FCF0E946F4A2091FA033091F7
:102F1000FB03AC01421B530B9A0181E0283833417B
:102F200008F480E008958091F9038695869586954A
:102F300008958091F903877008950E946F4A209147
:102F4000F7033091F803821B930B8838934138F0D4
:102F50008091F903002482FF0394802D089580E07E
:102F600008959091F903977081E0911101C080E07C
:102F7000089580912704089590912704982B9093A9
:102F800027040895982F9095809127048923809392
:102F90002704089510922704089580912604089527
:102FA00090912604982B909326040895982F90953D
:102FB0008091260489238093260408958093260413
:102FC00008951092260408958091FD0308950895B0
:102FD000FECF0895982F8091FC03282F29232917CD
:102FE00021F0892B8093FC03F3CF08959091FC038B
:102FF000292F2823211529F0809589238093FC030C
:10300000E7CF08950895FECF0895CF93C82F8091FC
:10301000FD038C238C1769F00E946F4A9093FB0389
:103020008093FA038091FD038C2B8093FD038C2FFA
:10303000EADFCF9108959091FD03292F28232115D0
:1030400079F0809589238093FD03811551F00E94CA
:103050006F4A8093FA039093FB038091FD03D3CFD3
:10306000089580E090E0F5CF8091FD03811541F057
:103070001092FD031092FB031092FA0380E0C3CF7D
:103080000895CF93C091270480912604C82B809186
:10309000FD03811551F037DF8111E6DF8091FD03DB
:1030A000C82B0E9467488111DFDF8C2FCF910895D4
:1030B000CF93DF93C0910601D0910701E2DF8883AF
:1030C000C0910601D091070148E050E06FEE73E037
:1030D000CE010E947955892B59F088E0FE01AFEEB0
:1030E000B3E001900D928A95E1F7CE010E94D74797
:1030F000DF91CF910895CF93DF93C0910401D091D8
:103100000501BFDF8983C0910401D091050140E230
:1031100050E06FEC73E0CE010E947955892B59F095
:1031200080E2FE01AFECB3E001900D928A95E1F7E9
:10313000CE010E94E447DF91CF9108950E94BF47DE
:10314000811529F08091F70987FF01C0D4CFB0CF56
:103150000895FECF0895962F2091F80922FF14C0FC
:10316000682F660F660F660F692B6093F903D4DA38
:103170000E946F4A9093F8038093F7038091F903BC
:10318000869586958695E5CFC7CA1092F903109269
:10319000F8031092F70380E0DCCF9091F90380955B
:1031A00089238093F903282F277021110BC08917D9
:1031B00049F09091F80992FF05C08695869586950D
:1031C000B5DAE3CF08959091F80992FB222720F910
:1031D000281749F080FB92F99093F80987EF99E05E
:1031E0004AD082E0DACF08958091F809002482FF66
:1031F0000394802DE8CF81E0E6CF80E0E4CF60E06B
:1032000070E0CB0153C460E070E0CB0149D4F7CF4C
:10321000A4E0B0E0EEE0F9E10C94B1548AD395D388
:103220001C82CE010496A8D381E080937B03AED3A9
:10323000198284E18A83CE010196B9D31B82CE0123
:103240000396C7D331D70E94FE45DDDF2496E2E026
:103250000C94CD54DDCF08957EC308956BD38111B6
:103260000C94B44508957DC308958CC308958EC30E
:10327000089591C308959BC30895A0C30895A9C359
:103280000895ADC30895ECC3089516C40895A6E04B
:10329000B0E0EDE4F9E10C94AF540E946F4A8C0168
:1032A00080912804909129048017910779F0198260
:1032B0001A820E946F4ABC0149815A8180E090E0E5
:1032C0000E948D0F10932904009328042696E4E0B1
:1032D0000C94CB540E947B4A609342047093430445
:1032E000809344049093450460933E0470933F049C
:1032F000809340049093410408950895089508959B
:10330000FEDF0C94B50C0895FECF08950895FEDFFE
:10331000FBCF88E19EE4B9D50E943129EFDFF0CFE1
:1033200081E0089581E00895FBCF08950895089500
:103330000895FCDFFCDFFCCF91DF811101C08ADF43
:1033400086E494E090DF87EF99E093DF0E9463309A
:103350008CDFC0D980917A03CDC90E94664A0E9451
:103360000A46EDD4E9DF0E94670F0E942C2880E016
:103370000E943F2D0E9406260E94F524C8CF0E947D
:103380004C450E9414330E9499310C94543DAAE09C
:10339000B0E0EDECF9E10C94A254C4DF982E811159
:1033A00014C075DF912CEBDF0E94CB250E9489278A
:1033B0000E94D42F91100E94842E0E9446400E94A9
:1033C000750F2A96E1E10C94BE54CBD42AE2A22ECA
:1033D00024E0B22E8501F12CD8014D905D906D90C6
:1033E0007D908D018F2D95D3462F572FBC01F394DF
:1033F000B5E0FB1609F468C0441655066606770664
:1034000059F38091460481FD8FD38EDF382E10E072
:1034100088248394812F7DD36B017C01F501419039
:103420005190619071905F01C414D504E604F704D3
:1034300009F444C0D701C60184259525A625B725E2
:103440008F839887A987BA8700E0412C512C3201DD
:1034500043948F819885A985BA8584219521A621D9
:10346000B721892B8A2B8B2BE9F03114D9F00983F2
:103470001A830E946F4A9C838B838D8221E0D7013F
:10348000C60184219521A621B721892B8A2B8B2B5C
:1034900009F420E049815A816B817C818D81922FD2
:1034A0000E948D0F0F5F440C551C661C771C033166
:1034B00081F6F501F292E292D292C2921F5F15302C
:1034C00009F0A8CF07DF6FCF4416550666067706CA
:1034D00009F097CF66CF1F93CF93DF9325D1EC01EF
:1034E000811522E5920708F05AC0811540E594073E
:1034F00008F0D7C0803E910528F58D3C910508F075
:10350000A9C0883A910578F4853A910508F09FC0E2
:103510008130910509F43EC00497813A9105D0F1BC
:10352000C0E0D0E037C0885A91094B97C8F7C85A15
:10353000D0E0CC0FDD1FCA58DE4F0990D881C02DD6
:10354000D46428C0811550E49507E8F4C11580E2E1
:10355000D80708F0BCC0C83ED105E0F0CE019A956E
:1035600081159F41E8F68D2F83D1182FCE01992721
:10357000DBD0212F30E0322F2227E901CC27DF7169
:10358000C82BD92B07C09927CFD0CC27DF70C82BE9
:10359000D92BD06ACE01DF91CF911F910895803849
:1035A00042E59407C8F5803652E5950708F05BC000
:1035B000C03482E5D807D0F4C03292E5D90708F0CC
:1035C0004BC08C2F8695869520E2829FC0011124E6
:1035D000C37021E030E0A90102C0440F551FCA9515
:1035E000E2F7EA01C82BD92BDD68D4CF8C2F869562
:1035F0008695877050E2859FC0011124C37021E039
:1036000030E0A90102C0440F551FCA95E2F7EA0154
:10361000C82BD92BDC68BECF803C52E5950758F407
:103620008F71C03AD245A0F590E0982F8827EC0121
:10363000C46FD06AAFCF805C9245809708F070CF9E
:10364000DC2FCC27CC27DF71C06FD06AA3CFA49723
:10365000D064A0CFD0659ECFCF71D0E0DC2FCC2737
:10366000C16FD06A97CF86958695877020E2829F3A
:10367000C0011124C37021E030E0A90102C0440F51
:10368000551FCA95E2F7EA01C82BD92BDA6882CF19
:10369000EFD0C82FD0E0DC2FCC27CC27DF71D06251
:1036A00079CF8F71E5D053E0CC0FDD1F5A95E1F74C
:1036B000CC27DF70282F30E084FF05C050E1859FC4
:1036C000900111243327C22BD32BD06963CF8D2FC8
:1036D0008F71CED0182FCE01992726D0212F30E020
:1036E000322F222722273F71282B392BE901D7CFF0
:1036F000462F672F2091FC083091FD08232B79F489
:10370000703F39F4403F59F480916A0B90916B0BF4
:103710000895753020F4433110F40C94153980E08D
:1037200090E00895E5DFD7CE803E9105D9F1C8F449
:103730008133910509F482C048F48932910509F476
:1037400072C08A32910509F480C0089589339105C9
:10375000E9F082389105D1F08533910509F45EC016
:103760000895843E9105D9F148F4823E910539F1DE
:10377000833E910549F181EE90E00895863E9105E2
:10378000C9F1873E910509F43EC008952091F709DB
:103790002370211164C02091F80923FF14C089E22D
:1037A00090E008952091F70920FD45C03091F80977
:1037B00030FF09C024FD24C083EE90E008952091DD
:1037C000F70922FDF7CF08952091F70922FD44C0A3
:1037D0003091F80930FD43C024FFF5CF11C020918E
:1037E000F80921FFF0CF8091F70984FD09C087EE29
:1037F00090E008952091F70923FFE5CF24FFF7CF4C
:1038000080E090E008952091F70923FD2BC03091CE
:10381000F80931FFE1CF84EE90E008952091F70997
:1038200025FFD1CFBCCF2091F70925FD1EC02091E7
:10383000F80923FFC8CF89E390E008952091F709A4
:1038400026FFC1CF8AE290E008952091F70926FF74
:10385000BACF81E390E0089582EE90E0089580EE83
:1038600090E0089586EE90E0089585E390E0089555
:103870009091F70992FF10C041E0282F2471243065
:1038800009F040E031E0282F2871283009F030E0BD
:10389000431711F02CE0822793FF10C041E0282F3E
:1038A0002471243109F040E031E0282F28712831BB
:1038B00009F030E0431711F02CE082273091F8092D
:1038C00030FF10C051E0282F2171213009F050E065
:1038D00041E0282F2871283009F040E0541711F0FA
:1038E00029E0822731FF10C041E0282F21712131CA
:1038F00009F040E031E0282F2871283109F030E04C
:10390000431711F029E0822794FD877E0895CF9315
:103910009C01FB01805E9245C1E0809738F4C5812F
:10392000C11104C0822F8F710E94040E8C2FCF9181
:103930000895089580E090E00E94B3559C0181E0D5
:10394000233E3E4F09F080E0089563EE7EEF80E075
:1039500090E00C94E1556FEF7FEF80E090E00C94E5
:10396000E155CF93DF93EC0182E090E00E94A655F1
:103970008883DF91CF910895FC01608182E090E01F
:103980000C94C75583E090E00C94A655682F83E013
:1039900090E00C94C755CF93DF93EC0184E090E066
:1039A0000E94B35599838883DF91CF910895FC01DC
:1039B0006081718184E090E00C94E155CF93DF93B6
:1039C000EC0186E090E00E94A6558883DF91CF91BC
:1039D0000895FC01608186E090E00C94C7558F92B9
:1039E0009F92AF92BF92CF92DF92EF92FF920F938E
:1039F000CF93DF93EC0188E090E00E94AE554B013D
:103A00005C0168839982AA82BB821C821D821E820D
:103A10001F8283E290E00E94A655282F30E040E00C
:103A200050E060E070E080E090E000E20E94D85456
:103A3000282939294A295B29288339834A835B83CA
:103A40006C837D838E839F83DF91CF910F91FF9055
:103A5000EF90DF90CF90BF90AF909F908F900895A0
:103A60000F93CF93DF93EC01488159816A817B8169
:103A700088E090E00E94D955288139814A815B8194
:103A80006C817D818E819F8100E20E94F354622FC0
:103A900083E290E00E94C755DF91CF910F91089586
:103AA000AB01BC018FE090E00C94D955AB01BC0197
:103AB00083E190E00C94D955682F8EE090E00C944F
:103AC000C7550895FECF08950895FECF0895962F07
:103AD00024E0829FF0011124E35FF54F41E050E0C4
:103AE00060E070E004C0440F551F661F771F9A9571
:103AF000D2F780819181A281B38184239523A6236B
:103B0000B72321E0892B8A2B8B2B09F420E0822F0D
:103B1000089594E0899FF0011124E35FF54F6081DF
:103B20007181828193810895A0E0B0E0EAE9FDE12E
:103B30000C94A7548CE692E09F938F930E94AC0C58
:103B40008DE0E82E8AE0F82E0F900F90812C912CBA
:103B500097E6A92E92E0B92E24E6C22E22E0D22EBC
:103B60000DE512E0CBE5D2E09F928F92BF92AF922B
:103B70000E94AC0CDF92CF920E94AC0CF7016191D5
:103B80007191819191917F010E942C0F9F938F934E
:103B90007F936F931F930F930E94AC0CDF93CF938F
:103BA0000E94AC0C9FEF891A990AEDB7FEB73E96BA
:103BB0000FB6F894FEBF0FBEEDBFF5E08F1691046F
:103BC00099F6CDB7DEB7ECE00C94C35480EA8A9541
:103BD000F1F7089500C00895F9CF0895F894E82FFB
:103BE000E295EF70F0E041A18F7021E030E0B90183
:103BF00002C0660F771F8A95E2F7CB01962F90954A
:103C0000942391A392A1892B82A378940895CF93B2
:103C1000DF93CFEBD1E089918F3F09F0DFDF81E0C7
:103C2000C43CD807C1F7CCEAD1E089918F3F09F0B5
:103C3000D5DF81E0CF3BD807C1F7DF91CF91089561
:103C40008F929F92AF92BF92DF92EF92FF920F936B
:103C50001F93CF93DF93EC01D62E062F10E0C801FF
:103C600081549E4F7C01FC0120812F3F09F45BC0F1
:103C7000F894E22FE295EF70F0E031A12F7081E02F
:103C800090E001C0880F2A95EAF7932F982B91A313
:103C900092A18095892382A378949CDFECEAF1E0DD
:103CA00041E050E060E070E0812C912C5401819162
:103CB0008F3F89F0A82FA295AF70A05EB0E02C9145
:103CC00030E08F7002C0359527958A95E2F7DB01C9
:103CD000CA0120FF04C080E090E0A0E0B0E0882AA4
:103CE000992AAA2ABB2A440F551F661F771F81E015
:103CF000EF3BF807E1F6F70180818F3F09F06EDFB7
:103D000061E081149104A104B10409F460E08D2DF7
:103D100063DF000F111F000F111FC00FD11F88821A
:103D20009982AA82BB82DF91CF911F910F91FF9060
:103D3000EF90DF90BF90AF909F908F90089567DFD6
:103D400084E1EDE0FAE0DF01982F1D929A95E9F702
:103D5000E9EFF9E0DF011D928A95E9F785E03BD0B4
:103D6000B1CEA4E1B0E0E7EBFEE10C94AE54FE016D
:103D7000319684E1DF011D928A95E9F710E0FE2E6D
:103D80000F2F612F8F2D902F5BDF1F5F1530C9F72D
:103D900044E150E06F2D702F89EF99E00E94795532
:103DA00021E0892B71F420E045E06DE07AE089EFB5
:103DB00099E012D0182F89DE812F6496E5E00C94EB
:103DC000CA5484E1EF2DF02FA9EFB9E001900D92D4
:103DD0008A95E1F7E9CF0895A0E0B0E0E2EFFEE1D7
:103DE0000C94AB54D82EE92EF62ED72F042FC22FC9
:103DF000211579F081E0809349040E946F4A9093E5
:103E000048048093470480E0CDB7DEB7E8E00C9427
:103E1000C754C0904904C114B1F3809147049091F4
:103E200048040E94004A059770F384E0089F8001CF
:103E30001124A8016D2D7E2D8F2D9D2F0E94795567
:103E4000892B41F0A8016D2D7E2D8F2D9D2F0E9475
:103E50008655CC2D109249048C2FD6CF98CA089540
:103E60000E94094A0E94794E54DA0E94914E75DAF6
:103E70000E949A4E0E949D4EF1DF0E94B34E0E9416
:103E8000934C0E94C04C55DAF5CF90934F0380932A
:103E90004E030895CF93DF93EC01FB0185818111DF
:103EA00004C081E0DF91CF91089563D88272FE0152
:103EB000E052F847EB30F105A0F7E45DF94A0C94C5
:103EC0005C548BD580E0EECF811521F07AD5FACF06
:103ED0008115E1F36BD5F6CF811521F03FD2F2CFFA
:103EE0008115E1F331D2EECF811521F051D2EACF25
:103EF0008115E1F340D2E6CF811521F063D2E2CF04
:103F00008115E1F352D2DECF811521F0FDD0DACF59
:103F10008115E1F3EAD0D6CFCF92DF92EF92FF92F4
:103F20001F93CF93DF93172FE82F711111C0411505
:103F300021F0F0E0E35DFB4FE4916E2F7E2F8E2F9A
:103F4000DF91CF911F91FF90EF90DF90CF90089578
:103F5000C62ED12CE72EF12C411521F0F0E0E35DC7
:103F6000FB4FE49186E0689F90011124CFEFD0E0F1
:103F7000C901BE010E941354AB01C601880F991FED
:103F8000F5E5F49FB001F59F700D1124861B970B8A
:103F9000682F660F680F6E01CE18DF08EC9DD00108
:103FA000ED9DB00D11249B2F169F60011124CD2C87
:103FB000DD247E01EC18FD086701EC9D7001ED9D8C
:103FC000F00C11246E01C61AD108B601169F6001CB
:103FD000179FD00C1124CD2CDD24CC19DD09EC9FCA
:103FE0006001ED9FD00C11247D2D43305105C1F0AF
:103FF0002C3F334050F441305105B1F0423051056F
:1040000061F47E2FEB2F9D2D08C04430510579F0CF
:104010004630510511F07B2F9F2D6E2FE92F8FCF4A
:104020007F2D9E2FEB2FF9CF7E2FEF2DF6CF9E2FDA
:10403000ED2D7B2FF2CF41E06FCF0895FCCF089597
:1040400090910B01291B922FE091F101F091F20167
:10405000242F462F682F892F90E009950895CF933C
:10406000DF93982F762F842FD22FC32F692FE6DF6F
:10407000962F672F482F2D2F3C2F892FE1DFDF91BF
:10408000CF9108958091210A843028F48370846050
:104090008093210A08958C3AE8F38370886AF8CFF8
:1040A000F1DF81E29AE0EFC8E1E2FAE085E08083A7
:1040B00011828FEF828383831482CF01E4C88091C1
:1040C000210A80FF03C086958695089580E00895B3
:1040D0009091250A933018F49F5F9093250A8115DB
:1040E00019F081E29AE0CFC8089581E0F1CF909174
:1040F000250A911519F091509093250A811519F010
:1041000081E29AE0C0C8089581E0F1CF8091250A4C
:1041100008958093250A08958091220A0895809138
:10412000230A08958091240A08950F931F93CF9333
:104130008091210A80FF09C0E091F501F091F6011C
:104140000995CF911F910F910895C0910D01009194
:10415000F1011091F20180910E01C81768F780916A
:104160000B019C2F981B892F20E040E060E090E03D
:10417000F8010995CF5FEFCFEF92FF920F931F9356
:10418000CF93DF93D82F162F042F8091210A80FF21
:104190000BC0C0910D01E090F101F090F20180910F
:1041A0000E01C81730F0C1DFCDB7DEB7E6E00C94E2
:1041B000C95480910B019C2F981B892F202F412FD0
:1041C0006D2F90E0F7010995CF5FE9CF982F762FFB
:1041D000842F2091210A20FF07C0692F2FDF962FFF
:1041E000672F482F892FC8CF0895CF93DF93EC0115
:1041F000EC81F0E0E855FD4F4491E1E2FAE06281A4
:104200008181E4DF8C818F5F8C83DF91CF91089572
:10421000CF93DF93EC01E1E2FAE0438162818C818C
:10422000D5DF8C818F5F8C83DF91CF910895CF9301
:10423000DF93EC012091240A9C81892F817090FDED
:10424000822F692F627091FD622F492F447092FD79
:10425000422F92DF8C8190E00196877099278C83A2
:10426000DF91CF910895A0E0B0E0E9E3F1E20C9492
:10427000AC54D82F062F142FE22E9091210A90FFD4
:1042800022C0E92FE695E695AE2FB0E0AC53BE4FC5
:104290008C918093E9049C7F9430D1F46D2F702F22
:1042A000842FCCDE962F672F482F892F65DFD09380
:1042B000220A0093230A1093240AE11421F081E2D8
:1042C0009AE00E944319CDB7DEB7E7E00C94C854DA
:1042D000823019F41091240AEACF863019F4D09173
:1042E000220AE5CF8930D9F3893109F7E9518E2FB8
:1042F0008170D82EE695F0E0E855FC4FC491F12C82
:1043000060910F01F61610F010DFD1CFFC9EC001B6
:10431000112470E00E9413548D2FD1100BC0860F12
:1043200020910D012F0D3327331F412F602F97DE72
:10433000F394E6CF861BF4CF282FE1E2FAE08181E7
:10434000438162818B5F8FCF81E0F6CF282FE1E23E
:10435000FAE0818143816281855085CF81E0F6CF8B
:10436000282FE1E2FAE062813AE0630F08F46FEF90
:104370004381818178CF81E0F3CF282FE1E2FAE019
:1043800062813AE0631B08F460E0438181816BCF76
:1043900081E0F3CF282FE1E2FAE043813AE0430FD6
:1043A00008F44FEF628181815ECF81E0F3CF282F47
:1043B000E1E2FAE043813AE0431B08F440E0628125
:1043C000818151CF81E0F3CF20E04DCFEF92FF927A
:1043D0001F93CF93DF93EC0110E0EE24EA94F12CCD
:1043E00060910F01161768F0A0DE8C819A8190FF12
:1043F0001DC08F5F8C83DF91CF911F91FF90EF9055
:10440000089520910D01210F3327331F70E0C7015C
:104410000E942754962F8C814091240A6091230A90
:10442000199F800D11241BDE1F5FDACF8150E2CF70
:10443000A0E0B0E0EEE1F2E20C94AA54FC0182812B
:10444000D1E080FDDFEFC0E0C090F101D090F2013B
:1044500080910F01C81790F068DE80914B04D13035
:1044600009F04BC0811102C080910F0181508093EF
:104470004B04CDB7DEB7E9E00C94C65480910D0132
:1044800090910B01891B8C0F20E040E060E090E0F0
:10449000F601099504E010E0B12CEC2EF12C80918E
:1044A0004B048B0D8F311CF16EE10E940654892F55
:1044B000082E001C00088E150F0499F480910D0140
:1044C0009701280F311D4091240A0403A0011124F3
:1044D00055954795559547956091230A8091220AF5
:1044E000BEDDBD0E01501040D1F6CF5FB1CF87FFCA
:1044F000DFCF90910F01890FDBCF90E001966091A3
:104500000F0170E00E942754B2CF0F931F93CF93F7
:10451000DF93C0910D010091F1011091F2018091A2
:104520000E01C81750F110E0C091F101D091F201D5
:1045300060910F01161770F1F8DD809109019091DB
:104540004A04980F90934A0420910A01280F20935F
:104550000A01121654F420910F012150330B092E39
:10456000001C0008921703061CF081958093090136
:10457000DF91CF911F910F91089580910B019C2F96
:10458000981B892F20E040E060E090E0F801099559
:10459000CF5FC5CFE12FF0E070E0CF010E9427543C
:1045A00020910D01820F90914A04092E001C0008F1
:1045B000E917F0059CF090910A01092E001C0008F3
:1045C0009E170F065CF0282F30E04091240A60917E
:1045D000230A8091220A43DD1F5FAACF90910B012D
:1045E000891B20E040E060E090E0FE010995F4CFF7
:1045F000A6E0B0E0EEEFF2E20C94AB548D839E8324
:10460000AD81BE811496FC912F2F30E0D9010E941C
:1046100082549B01AC010E9497546B017C0180E2A3
:1046200090E09C012F1B3109F901A5E5B0E0A7013D
:1046300096010E94975469837A838B839C839F01A0
:10464000DF010E947C549B010E9491549B01AC01AC
:104650002C0D3D1D4E1D5F1D69817A818B819C81D2
:104660000E943A54022F30E00A3240F5A901440F6B
:10467000551F420F531F55954795142F1095F12C38
:1046800085E5E82EE01A80910F01F81628F14DDD3E
:10469000AD81BE8114969C9181E0911519F0903204
:1046A00019F48FEF8093080180910801890FED8143
:1046B000FE8184832696E8E00C94C75485E590E05B
:1046C000821B930BAC01440F551F480F591F57FF16
:1046D000D2CF4F5F5F4FCFCF8E2DF1FC802F209137
:1046E0000D012F0D3327331F412F6091230AB7DCB3
:1046F000F394C9CF0F931F93CF93DF93EC0100E0A6
:1047000010E090910F010917110564F00EDD8C8106
:1047100090E00196817099278C83DF91CF911F9152
:104720000F9108954C8180910D019801280F311D42
:104730006091230A8091220A96950917110544F485
:10474000411541F04091240A8ADC0F5F1F4FD9CFF9
:104750004115C1F340E0F8CFA0E0B0E0E2EBF3E2B6
:104760000C94A354FC016280448081E08483E8EAD5
:10477000F2E07490E7E2F3E0E491C091240AC69578
:10478000C158D0E0CC0FDD1FCD2FDD27812C25E0D7
:10479000922EAA24AA94B12C55245A94E719EE2EED
:1047A000F12C80910F01881630F0BFDCCDB7DEB759
:1047B000E0E10C94BF54C82CD12C83E0681658F467
:1047C000989CF0011124E45BFB4F8091220A8083C6
:1047D0008091230A818341101BC09C9CF0019D9C09
:1047E000F00D1124E45BFB4F1382128280910D01C6
:1047F0009601280F311D9C9CF0019D9CF00D112409
:10480000E45BFB4F42816181808129DC8394C9CFC5
:104810009C9C80019D9C100D1124045B1B4FF80192
:1048200083818115F1F081508383589EC00111244A
:10483000648170E00E941354FB01FF27E855FD4F8F
:104840008491E82FE7195E9EC0011124B7010E94F0
:1048500013548091240A689FB0011124F8017283D7
:10486000C5CF0E945555B5010E9427548C179D074E
:104870000CF0BCCFF3E06F1698F00E945555B501CF
:104880000E942754F80180830E9455552091230AE5
:104890002695622F70E00E942754280FF80121838B
:1048A0009C9CF0019D9CF00D1124E45BFB4F128257
:1048B0008091240A893C58F088EC9C9CF0019D9CD6
:1048C000F00D1124E45BFB4F848383838FCF84310D
:1048D000A0F784E1F2CFE1E2FAE080818E7F80836D
:1048E000CF010E9443191092EA041FCCE1E2FAE0E2
:1048F00080818E7F80831092EA0417CC6091210A18
:104900006695669570E04BE050E080E191E00E9492
:104910006C55892B19F481E08093EA040E946F4A58
:104920009093E3048093E20408959091210A90FF0C
:104930002CC0811559F18B3258F58F73880F880F71
:104940009091210A9370892B8093210A611521F09F
:1049500081E29AE00E9443196091210A669566956A
:1049600070E04BE050E080E191E00E946C55892BB3
:1049700089F01092EA0481E08093E5044091240AD2
:104980006091230A8091220A1FCD089581E0D6CF3D
:104990008AE2D4CFB3DFEFCF682F8091210A8695CA
:1049A00086958F5F8B3208F081E0BFCF81E0F4CF36
:1049B000682F8091210A869586958A9509F48AE266
:1049C000B4CF81E0F5CF61E0B0CFE1E2FAE08081E1
:1049D0008160808386958695F6CF8091210A80FF3D
:1049E00001C079CFF2CF60E0A0CF8091E8048111BF
:1049F0001FC081E29AE00E9441198091210A84300F
:104A000028F452DB81E29AE00E9441193BDB1092CC
:104A1000EA04E091EF01F091F00109958091210AFB
:104A200080FF03C086958695DEDF81E08093E804F1
:104A30000895E1E2FAE08081816080838695869521
:104A4000D2CF0F931F93CF93DF938091EA04811508
:104A500009F441C08091E904E091210AE695E695C8
:104A6000E81BE093E404853109F48BC008F044C0EE
:104A7000893009F47CC0A0F5823009F466C0863024
:104A800009F46CC0C0EDD7E00DE110E28091E504BF
:104A9000811561F01092E5040E946F4A9093E3043F
:104AA0008093E2041092E7041092E6040E946F4A99
:104AB0002091E2043091E304821B930B8F3F9F47C8
:104AC00050F42C0F3D1F3093E3042093E20482EE58
:104AD00094E0F8010995DF91CF911F910F9108950E
:104AE0008F3081F6E695F0E0E556FD4FE491CE2F4C
:104AF000D0E008E112E2CACFC4EFD1E00AE713E246
:104B0000843221F288F4C8E2D0E008EF12E2883162
:104B100009F4BCCF833209F0B5CFE6E9F2E0C591E4
:104B2000D59107E111E2B2CF853209F0ABCF8E2FDC
:104B300063E00E94FA53E92FF0E0ED56FD4FE49157
:104B4000CE2FD0E00CEA13E2A1CFF0E0EC55FD4F00
:104B5000E491CE2FD0E005EF10E298CFF0E0EF55D2
:104B6000FD4FE491CE2FD0E008E011E28FCFE69523
:104B7000F0E0E256FD4FE491CE2FD0E006EE11E2D8
:104B800085CFF0E0E856FD4FE491CE2FD0E005E868
:104B900012E27CCF089555CF089589E29AE00C94F3
:104BA0003F198DE18093290A89E29AE00C943F191C
:104BB0008091290A86958695869508958091290A7F
:104BC00081FD08C082608093290A89E29AE00E94F0
:104BD0003F19A0C108958091290A81FF08C08D7FE7
:104BE0008093290A89E29AE00E943F199FC10895A3
:104BF0008091290A81FF01C0EECFE0CF8091290A80
:104C000086958170089580911B01089589E29AE04C
:104C10000E943D198091290A82FFC3DF8091290AF1
:104C2000803220F0877088618093290A9091290A48
:104C3000892F817090FF04C0892F8695869586956F
:104C400045C19091290A892F869586958695983138
:104C500040F48F5F880F880F880F9770892B80939F
:104C6000290A8091290A81608093290A89E29AE0C1
:104C70000E943F198091290A86958695869526C1BE
:104C80008091290A883088F088508093290A91E021
:104C9000883008F490E08091290A90FB80F9809395
:104CA000290A89E29AE00E943F198091290A869593
:104CB000869586950BC18091290A80FD12C081607E
:104CC0008093290A813019F489E08093290A89E2C6
:104CD0009AE00E943F198091290A869586958695CB
:104CE000F5C008958091290A80FF09C08E7F8093C6
:104CF000290A89E29AE00E943F1980E0E7C00895FE
:104D00008091290A80FF01C0EDCFD5CF8091290A7B
:104D10008695869586958F5F8F71843008F080E048
:104D2000880F880F880F9091290A9770892B80939C
:104D3000290A91E0883008F490E08091290A90FBDC
:104D400080F98093290A89E29AE00E943F198091B4
:104D5000290A869586958695B9C0843008F083E047
:104D60002091290A2770982F990F990F990F922B4C
:104D70009093290A21E0983008F420E09091290AC4
:104D800020FB90F99093290AA1C0E7DF89E29AE01D
:104D90000C943F19FC01DB0115968C918115C1F033
:104DA000F857E730F105A8F4E95CF94A0C945C5433
:104DB00083E0EBDF80E0089580E0FBCF61DFFACF96
:104DC00040DFF8CF9DDFF6CFA1DFF4CF11DFF2CFC8
:104DD00081E00895A0E0B0E0E0EFF6E20C94A75483
:104DE0008C0180918600909187006CE070E00E94B9
:104DF00013546017710768F0C80169E070E00E9401
:104E00001354262F972F822FCDB7DEB7ECE00C94EA
:104E1000C3548091860090918700E0908600F090C6
:104E20008700C0908600D0908700C6E0D0E0BE0129
:104E30000E94135420E030E0060F171F211D311D82
:104E40004801590185E0880C991CAA1CBB1C8A9555
:104E5000D1F7C701BE010E941354E12CF12CA70128
:104E60009601260F371F411D511DC501B4010E9437
:104E70003A5469017A01E0918600F0918700CA01F5
:104E8000B9010E94EB539B01AC01DF010E949754D2
:104E90009B01AC01C701B6010E94EB53DC01CB01C1
:104EA0002FE0B695A795979587952A95D1F72091EC
:104EB000860030918700281739071A061B0620F450
:104EC0008091860090918700282F9DCF8430E0F458
:104ED00081111BC0909180009F7D90938000209154
:104EE000860030918700A82FB0E00E94825423E012
:104EF00030E040E050E00E943A54C9016BDF9093EB
:104F00008B0080938A00089583E0909180009062E6
:104F1000E4CF08951092EC041092EB041092ED048B
:104F2000EFE6F0E08081816080830895EFE6F0E0B5
:104F300080818E7F80833CDEC9CF1F920F920FB697
:104F40000F9211240BB60F92EF92FF920F931F93C3
:104F50002F933F934F935F936F937F938F939F9381
:104F6000AF93BF93CF93EF93FF9380911C01823057
:104F7000D9F08F5F80931C01FF91EF91CF91BF918A
:104F8000AF919F918F917F916F915F914F913F91E1
:104F90002F911F910F91FF90EF900F900BBE0F90EC
:104FA0000FBE0F901F90189581E080931C012BDE9F
:104FB000C82F0091EB041091EC040F5F1F4F23DE0C
:104FC00028E7289FB0011124C8010E941354909330
:104FD000EC048093EB042C9FB0011124660F672F23
:104FE000661F770B71950E94135467FD6FE78091E0
:104FF000ED04823069F5603429F480916F008E7F72
:1050000080936F00E62FF0E0E355FC4FC491E090F1
:105010008600F0908700CCDD182F2C2F30E0D701D0
:105020000E9482542FEF30E040E050E00E943A545A
:10503000C90163E070E00E941354169FC001179FDE
:10504000900D1124C7DE90938B0080938A0094CF3B
:105050008130C1F66F37D0CF269A2E9882E28093A6
:10506000800089E1809381008FEF9FEF909387000C
:1050700080938600CBDDC2DD81114CCF08950C9466
:105080005A48089581152CE7920741F42091FE08B3
:105090003091FF08232B11F480E090E00895EEECAE
:1050A000F6E080E090E06EEE7BE24CE75BE224E22B
:1050B0003BE27783668351874087338722879787D0
:1050C0008687019670968032910599F70895FB01C5
:1050D000811520E2920728F4811541E0940738F405
:1050E00008959C0130522115304348F00895392F1E
:1050F00094FF02C03295307F2081232B2083992793
:105100000895462B22FF0FC0982F92959F708F70A5
:10511000892B962F92959F706F70692B942F929583
:105120009F704F70492B982F9623961309C050E01B
:105130004095509590E04823592381E0452B09F094
:1051400080E00895CF92DF92EF92FF921F93CF936A
:10515000DF93CDB7DEB72A970FB6F894DEBF0FBE48
:10516000CDBFEAE2FAE080E491E0DF019C011D920C
:1051700021503040E1F7EEEEF5E080EEDF011D92C8
:105180008A95E9F78AE2C82E8AE0D82E7F0110E0DE
:10519000F701D182C082BE016F5F7F4F812F0E94D5
:1051A0007D38892B79F488E0FE013196D601019093
:1051B0000D928A95E1F789859A85D70113969C937C
:1051C0008E931297BAE0CB0ED11CE7E0EE0EF11CE5
:1051D0001F5F1032E9F62A960FB6F894DEBF0FBEB5
:1051E000CDBFDF91CF911F91FF90EF90DF90CF90D7
:1051F0000895A6E0B0E0EFEFF8E20C94AD540EEEA7
:1052000014E0F12C88E0E82EBE016F5F7F4F8F2DF8
:105210000E948138892BD9F4F8018E2D11928A953C
:10522000E9F7B8016C5F7F4F89819A8150DFF801FF
:1052300091838083B8016B5F7F4F8B819C8147DFB7
:10524000F801938382838D8186838E818783F39493
:10525000085F1F4FF0E2FF12D7CF2696E6E00C94CE
:10526000C9541DDF6FDFC5CFAAE0B0E0EAE3F9E281
:105270000C94AC548C01603239F5DC011196EC9140
:105280001197EE3008F5F0E0E25CF94A0C945C54BA
:1052900088E0E7EFF1E0DE01119601900D928A952A
:1052A000E1F7F80131968FE1DF011D928A95E9F768
:1052B00086E0F801808388E0FE013196D8011496DB
:1052C00001900D928A95E1F72A96E7E00C94C85474
:1052D0008CE78C9382E011968C93119712961C9216
:1052E000129713961C92F0CFFC0182819381092EB4
:1052F000000CAA0BBB0B45E0880F991FAA1FBB1F10
:105300004A95D1F7AC01BD01405E5F4F6F4F7F4FB3
:10531000481759076A077B07B8F28C37F2E09F07F6
:10532000A105B10588F64D3722E0520761057105E8
:1053300020F04CE752E060E070E0481B590BBC01E4
:10534000635D7A4FC8010E946355BECF4FE150E0C4
:105350006FEF70E001960E948F558091FE08D80192
:105360008C938091FC0811968C93119712961C9245
:10537000129713961C92139781E014968C931497AE
:105380008DE015968C93A0CF81E090E09093FD087E
:105390008093FC0882E390E09093FB088093FA08E6
:1053A0000E946F4A9093F9088093F8088DCF8091FE
:1053B000FC089091FD08892B91F160E080E00E944B
:1053C000671DE82E6DE081E00E94671DF82E809138
:1053D000F8089091F9080E94004A8536910550F12D
:1053E000E11441F1F11431F10E946F4A9093F908F0
:1053F0008093F8088091FA089091FB0801979093A8
:10540000FB088093FA08892B51F41092FD08109242
:10541000FC0881E090E09093FF088093FE08809163
:10542000FE08F80180838091FC0881838091FA084E
:1054300082834ACF82E390E09093FB088093FA083E
:10544000EECF1092FF081092FE083ECF40E250E0EF
:105450006FEF70E00E948F5537CF1296EC91129744
:10546000E93008F031CFF0E0E45BF94A0C945C5489
:10547000FC0131968FE1DF011D928A95E9F780E208
:10548000F80180838183838383E0878F1DCF139608
:105490008C913AE0D32EFE0131967F01DF01ED2D94
:1054A0001D92EA95E9F7B7010E947938D8018D93EA
:1054B000F70101900D92DA94E1F706CF1396FC9074
:1054C0008AE0F8013496DE01119601900D928A95DA
:1054D000E1F789819A81D6DD9A8389838B819C81CA
:1054E000D1DD9C838B838D819E81CCDD9E838D83DA
:1054F0008F819885C7DD98878F83BE016F5F7F4F4F
:105500008F2D0E947B38F8018083C9DDDDCE139694
:105510008C912AE0D22EFE0131967F01DF01ED2D24
:105520001D92EA95E9F7B7010E947D38BFCF139627
:10553000FC908AE0F8013496DE01119601900D92FC
:105540008A95E1F789859A859DDD9A878987BE01CD
:105550006F5F7F4F8F2D0E947F38F8018083F2DDCF
:10556000B3CE13968C9196E0D92EFE0131967F0131
:10557000DF01ED2D1D92EA95E9F7B7010E94813810
:1055800095CF1396FC9086E0F8013496DE011196D3
:1055900001900D928A95E1F789819A8173DD9A8352
:1055A00089838B819C816EDD9C838B83BE016F5FC1
:1055B0007F4F8F2D0E948338F80180831ADE84CEBE
:1055C000A6E0B0E0E6EEFAE20C94B15490936B0BD7
:1055D00080936A0B811520E2920730F40E94510DEE
:1055E0002696E2E00C94CD5480EF89838A830E9452
:1055F0006F4A8160BC0149815A8181E091E00E943B
:105600008D0FEECFA6E0B0E0E8E0FBE20C94B154E1
:1056100090936B0B80936A0B811520E2920730F414
:105620000E94650D2696E2E00C94CD5480EF8983AC
:105630008A830E946F4A8160BC0149815A8181E05E
:1056400090E00E948D0FEECF0F931F93CF93DF93C7
:105650008C01EB016EEC78E08C2F0E947938892B5D
:1056600071F4DD27C852D74F8881F8011282188261
:105670008330E9F048F4813059F0823081F0DF91D5
:10568000CF911F910F9108958430B1F08530B9F713
:105690008091CE089091CF08009789F306C0809141
:1056A000D0089091D108009799F3ACDFE8CF8091B2
:1056B000D2089091D308F7CF8091D4089091D50863
:1056C000009799F72091CE083091CF088091D008AB
:1056D0009091D10821153105F9F2009731F7C901F0
:1056E000E4CFCF93DF93D82FC92F6ADF8D2F9C2F64
:1056F00089DFDF91CF9108950F931F93CF93DF93AD
:105700008C01EB016EEC78E08C2F0E947938892BAC
:1057100009F057C0FE01FF27D80112968C9112970D
:10572000E852F74F8130A9F415968C9182FD4EC056
:1057300080FF4CC082E080838091D0089091D10896
:105740000097B9F48091CE089091CF080097C9F1E5
:1057500010C08230A1F515968C9182FD26C080FD87
:105760000AC083E080838091D2089091D30800978B
:10577000F1F026DF26C084E080838091D4089091E8
:10578000D5080097B1F78091CE089091CF08009787
:1057900001F1A7DF8091D0089091D108009749F7D7
:1057A0008091CE089091CF08E4CF85E080838091EE
:1057B000CE089091CF08009721F093DFF1CF86E0DB
:1057C0008083DF91CF911F910F91089581E08083B5
:1057D000B9CF8091D0089091D108B8CF0F931F9383
:1057E000CF93DF938C01862F6EEC78E00E9479389E
:1057F000892B91F4C091CE08D091CF08209761F009
:10580000F8018281833039F4CE016BDFCE0169DF8C
:10581000CE0167DF01C0E0F7DF91CF911F910F91BB
:105820000895AAE0B0E0E7E1FCE20C94B1549C01D9
:1058300097558115914030F088EC90E02A96E2E08F
:105840000C94CD54BE016F5F7F4F822F0E94793838
:10585000892B91F789859A85F1CF80E290E00895B0
:105860008032910540F424E0880F991F2A95E1F7D2
:105870008253994F089580E090E00895CF93DF938D
:10588000EC01FB018581811130C0D755C115F1E0D4
:10589000DF0758F56EEC78E08C2F0E947938892B61
:1058A00021F5CE0124E0880F991F2A95E1F7FC012C
:1058B000E253F94F22812130E1F42091CE0830915A
:1058C000CF08232B91F02091D0083091D108232BC1
:1058D00061F02091D2083091D3084091D4085091C2
:1058E000D508242B352B232B61F081E0DF91CF915C
:1058F00008952230D1F72091D2083091D308232B7C
:10590000A1F3FC01ED52F94F20812E7F20838253B9
:10591000994F0E94A244E9CFA1E0B0E0E2E9FCE2A5
:105920000C94A8546983BE016F5F7F4FD0DB5C018C
:105930000EEE14E0CC24CA94EE24E394F12CF8018A
:10594000D780D3FE49C0808191818A159B0599F447
:1059500094802D2D4681692D8981D3DB811559F0E5
:10596000892D0E94FB0EC81634F4F8019581E2805F
:10597000F380F92AC82EF801828193818A159B054C
:10598000A9F4D1FE13C095802D2D4681692D898102
:10599000B8DB811559F0892D0E94FB0EC81634F42E
:1059A000F8019481E080F180F92AC82ED0FE14C05D
:1059B000FFEFCF1211C081E0E816F10469F42D2D3C
:1059C000F801468160E089819CDB811529F0F801AE
:1059D0008581E280F380F82A085F1F4FF5E00E3ED4
:1059E0001F0709F0ACCFC7012196EBE00C94C4541B
:1059F000AB0124E630E0BC0188E70E945F4B9C01CC
:105A000081E0232B09F080E00895AB0124E630E02B
:105A1000BC0188E70E94A94B9C0181E0232B09F07F
:105A200080E008950F931F93AC019B0104E610E002
:105A300060E488E70E94F54B9C0181E0232B09F08C
:105A400080E01F910F9108950C942B4B08950895B9
:105A5000FECF0895ECE6FBE080E092E0DF019C01E0
:105A60001D9221503040E1F7F093710DE093700DDD
:105A70008FEF9FEF90932C0980932B090895CF937C
:105A8000E6DFE6DF90E280FF90E8809327099093BD
:105A90002609DADF6BE070E085EB98E0B6DF811174
:105AA0000CC089E998E09F938F930E94AC0C0F90F3
:105AB0000F90C0E08C2FCF9108958091270965E069
:105AC00070E081FD08C084E998E09FDF81110BC080
:105AD0008EE698E0E8CF89E698E097DF811103C071
:105AE00081E598E0E0CF6DE070E084E498E08DDF40
:105AF000C82F8DE298E0C115B1F20E947B4ADC010B
:105B0000CB01805A9541AF4FBF4F80936C0D90935E
:105B10006D0DA0936E0DB0936F0D9CDF81E08093AF
:105B20002A098093290910922809C4CF20912609B7
:105B300036E0839FC0011124269F800D911D112402
:105B4000811522E0920714F080E090E08459944F90
:105B50009093710D8093700D08952091700D309188
:105B6000710D26563B4040912609642F70E0C90113
:105B70000E941354481B463010F4240F311D211588
:105B800082E0380710F020E030E02459344F3093A1
:105B9000710D2093700D0895CF93DF93982FC62F2A
:105BA00081E09A3019F09D3029F480E06AD0DF91CD
:105BB000CF9108952091700D3091710D86E0F9011B
:105BC000A0E0B9E001900D928A95E1F7903EB0F027
:105BD00086E0F90111928A95E9F7C1111BC0C091C5
:105BE000700DD091710D46E050E0BE0180E099E06B
:105BF0000E947955892BE1F4B0DFD9CFF6E09F9F61
:105C0000B00111246054774F46E050E0C9010E9472
:105C10006355E3CFE091700DF091710D9F012A5F04
:105C20003F4F2E173F07D9F2808180958193F9CF9E
:105C3000CC56DB40CE0125E0969587952A95E1F775
:105C400021E030E0A90102C0440F551F8A95E2F718
:105C5000CA0140912B0950912C09842B952B259634
:105C600045E0D695C7954A95E1F702C0220F331F4C
:105C7000CA95E2F7822B932B90932C0980932B09E2
:105C8000BBCFCF93382FE091700DF091710DEC5692
:105C9000FB4020912609622F70E0CF010E9413542F
:105CA000281B822F311561F066E00E94FA53C82F3D
:105CB000C15010F4CF91089560E080E26DDFF8CF1D
:105CC0008E0F9F2F911D811522E0920710F080E02A
:105CD00090E08459944F9093710D8093700DEACFAA
:105CE0001F93CF93DF93EC01162FFE018491811156
:105CF00004C0DF91CF911F910895612F4DDF219650
:105D0000F4CFEEDF81E0BDCFCF93C0912A09C1115E
:105D100005C0C09129098C2FCF9108950E947B4A1C
:105D2000DC01CB01805A9541AF4FBF4F80936C0D82
:105D300090936D0DA0936E0DB0936F0D8091290916
:105D40008111E9CF62E070E084ED97E05EDE8111C1
:105D50000BC080EC97E09F938F930E94AC0CC09196
:105D600029090F900F90D7CF81E080932909D3CFD5
:105D7000A4E0B0E0EEEBFEE20C94A1548C838091A1
:105D80002B0990912C09892B09F456C080912A097E
:105D9000811509F451C08091280981114DC0B4DFEB
:105DA00010E01B8244244394512C00E247E0F42E7F
:105DB00020912B0930912C0921153105E9F111159C
:105DC00039F0FC81F11104C037C04B814F5F4B8328
:105DD0005B81852F90E0520102C0AA0CBB1C5A9532
:105DE000E2F7A50142235323452B79F3209127099C
:105DF00020FD26C09695879596958795282F9B819F
:105E00009295990F90763FE1390F90931F018093FF
:105E10002201309320012093230167E070E08DE19F
:105E200091E0E6DD811115C08AE098E09F938F93A1
:105E30000E94AC0C0F900F902496E2E10C94BD549C
:105E40009B81990F990F990F37E0390F80E023E07C
:105E5000DCCFBB81A0E2BA9FC001112420912709A9
:105E600020FD0AC060E270E08459944FDBDD8111AF
:105E700066C081EF97E0DACFE6E0F9E0202F1192DB
:105E80002A95E9F746E353E05A83498362E373E0D6
:105E9000E981FA81A191FA83E983FB012191BF0194
:105EA000280F392F311DA9014459544F1A01EA2FE7
:105EB000F0E0EA5FF64F20E030E06F2C621A842CAD
:105EC000022E01C0880C0A94EAF76101912CD601D8
:105ED000ED906D01E820462D4919477050E0BE2D28
:105EE000042E01C0BB0F0A94EAF77B2E5195419511
:105EF00051094770552701C0E6944A95EAF7EB2A05
:105F00004081E42AE082939448E09412E0CF2F5F2E
:105F10003F4F31962830310581F6AAE3B3E0E9819D
:105F2000FA81AE17BF0709F0B3CF60E270E086E0F8
:105F300099E078DD811103C086ED97E077CFA094DA
:105F4000B09480912B0990912C098A219B219093E8
:105F50002C0980932B091F5F2BCFCF93C0912A0967
:105F600080912909C11106C091E0C82FC9278C2F43
:105F7000CF9108958115D9F362E070E08EEB97E040
:105F800044DD81110BC089EA97E09F938F930E94B3
:105F9000AC0CC09129090F900F90E9CF10922909FC
:105FA000E6CF0C94BD0C08950F931F9380912A099E
:105FB0008115F1F060E080E0B9DDF3DF80E0D8DE4C
:105FC000809129098115A1F00E947B4A00916C0DF6
:105FD00010916D0D20916E0D30916F0D601B710B46
:105FE000820B930B6F3F7F4F8F4F9F4708F4B5DFB6
:105FF0001F910F910895579A0895FC01EE0FFF1F0E
:10600000E80FF91FEE58F24F618340832283089511
:10601000FF920F931F93CF93DF93182F062FF42E29
:10602000C0E0D0E02F2D402F612FCE01E6DF21967A
:10603000CE31D105B9F7CDB7DEB7E5E00C94CA543F
:106040003BB13F772BB120684FB7F89482E79DE0D2
:10605000FC010196508168E02BB9000000C057FF99
:106060003BB9550F000000C000C000C03BB900C0E4
:106070006A9591F75DE08C3C950751F74FBF8FE52E
:1060800094E00197F1F700C0000008950C942C19DA
:10609000089580E00E94891D862F817008950E94D6
:1060A000B11E2FEF86E791E0215080409040E1F74C
:1060B00000C000000E94B11EECDF811519F0E6DF80
:1060C0000C94AB4A0895EBCF08959C018D32910555
:1060D000F9F088F48832910548F44E97E0F42450A2
:1060E00031092A313105A0F080E0089581E02A329B
:1060F0003105D1F7089581E02D3292E0390709F09A
:1061000080E091E02C34310509F090E0892B08956E
:1061100082E00E94D01781E00895EF92FF920F93E2
:106120001F93CF93DF93EC017B0183372CE792071A
:1061300051F4FB01858181110DD180E0CDB7DEB72F
:10614000E6E00C94C954823AF2E59F07A1F150F4BD
:1061500090528115904210F1C13ED10561F1C53ECA
:10616000D10502C0823B924509F03EC085EE90E029
:106170008770992701E010E002C0000F111F8A9577
:10618000E2F7B9D090912D098115E9F0F7018581E9
:106190008115A1F0902B90932D09CFCFFB01868123
:1061A000803110F58D2F99278F71992782309105B5
:1061B00011F04297D9CF81EE90E0DACF0095092314
:1061C00000932D09BACF892F8023811569F0802F84
:1061D0008095892380932D09802F0E94C217F70193
:1061E0008581811509F4A9CF0E94B917182F0E9443
:1061F000E417082F80D0811102C081E09FCF72D0B8
:10620000F70185818115C9F3102B1D7911115BC030
:10621000C115F0E5DF07A0F4C11520E4D20708F0AE
:1062200058C0C63ED10549F3CE0190528115904227
:10623000E0F4F7018681803108F43EC0DD2715C007
:10624000C03EF2E5DF0750F5C03C22E5D207A8F6D4
:10625000C03A82E5D807E0F4C036E2E5DE0768F62A
:10626000CE0192558034910540F20E94E117CE0193
:106270002CDF811541F180912D09811531F00E94AB
:10628000CD1792E089270E94DE170E949E18B5CF95
:10629000C43BF2E5DF0709F4B0CFE7CFC9372CE7FD
:1062A000D20730F4C7378CE7D80708F0A6CFDDCF88
:1062B000CB37ECE7DE07EFCF8D2F8F71843109F4F8
:1062C0009CCF863161F029D080912D090E94BC17A6
:1062D00094CFF7018681803108F0B0CF8ECFC6EE23
:1062E000D2E1C3CF0E946F4A88579C4E90932F09EA
:1062F00080932E0908958091300908950895809122
:106300003009811109C00E94CA170E943418EADFBF
:1063100081E080933009F2CF089580913009811592
:1063200039F082E20E94FF121092300980E0E6CF3D
:10633000089580913009811561F00E946F4A209183
:106340002E0930912F09821B930B8F3F9F4708F432
:10635000E4CF089580913009811509F0DECFCFCFC9
:106360000895EF92FF920F931F93CF93DF93809145
:10637000A409E0913109CDE0811129C0CDB7DEB784
:10638000E6E00C94C954D1E0DE0FD0933109EE2E33
:10639000F12CCE9FF0011124E45CF64F848181152D
:1063A000A9F087819085892BD9F4818592858F3FCB
:1063B0009807B1F061E0D4DFCE9DF001CF9DF00DE4
:1063C0001124E45CF64F14820E94E117ED2F8091B6
:1063D000A409E817C0F21092A40910923109CECF97
:1063E00000811181228133814481558166817781C9
:1063F00080850E940017E0CF08951092A6091092A0
:10640000A509EEEEF5E08581811102C014821682A5
:10641000379686E0EE3CF807B1F70895AC0130916D
:106420003A0960913B09232F621301C00895822F1E
:1064300090E0FC01EE0FFF1FEE5CF64F0190F08143
:10644000E02DE417F50791F467E0649FF001659F84
:10645000F00D1124E251FA4F41E044832313E6CFBB
:1064600001968370992780933A0908950196282F01
:106470002370DACF6F927F929F92AF92BF92CF92AA
:10648000DF92EF92FF920F931F93CF93DF93DB0185
:1064900014962C911497211157C0A090A409ECE3F5
:1064A000F9E060E070E0B12C66246394712C6A1509
:1064B00008F049C0C384D484ED90FC9011972FEF6D
:1064C0003FEF912C492D50E08701090D111D090D59
:1064D000111DE801088119810115110539F0C01657
:1064E000D10609F0A90193949A01ECCF2F3F32070E
:1064F000D1F1E30102C0CC0FDD1F2A95E2F7BC2ADF
:10650000930102C0220F331F9A94E2F7A901415070
:106510005109B416150631F512962D913C91139739
:106520004DE0469FF001479FF00D1124E45CF64FCB
:106530003087278324E02483108211828187928709
:1065400021E015962C936ADFDF91CF911F910F9177
:10655000FF90EF90DF90CF90BF90AF909F907F9093
:106560006F90089514826F5F7F4F3D96A0CF1F9369
:10657000CF93DF93C0913A0917E080913B098C13C8
:1065800006C0EFDE3ADFDF91CF911F910895D0E092
:10659000FE01EE0FFF1FEE5CF64F80819181189F88
:1065A000B001199F700D112462517A4F63DF21965B
:1065B000C370E3CF0F931F93CF93DF93FC01CB0105
:1065C0000081118140E020E030E0D801A30FB11D2F
:1065D000A30FB11D6D917C9161157105C1F0DC01B6
:1065E000CD91DC9120E007C051E06A177B0709F0EC
:1065F00050E0452B2F5FDE01A20FB11DA20FB11D90
:106600000D90BC91A02D109779F73F5FDECF41151B
:1066100041F0231708F0CF01DF91CF911F910F9127
:10662000089580E090E0F8CF80912401811529F150
:106630008091A7099091A8090097F9F00E94004A5B
:106640002091A5093091A60928173907B0F4909137
:106650003A0980913B09981751F089DF1092A609F9
:106660001092A5091092A8091092A709089579DE41
:106670001092A8091092A709C0CE08951092A809F7
:106680001092A7091092240180913B0980933A0946
:10669000B4DE67CE80912401811509F0EFCF81E04F
:1066A000809324010895ABE0B0E0E9E5F3E30C94B6
:1066B000A1545C012B0180352CE7920769F4DB01C2
:1066C00015968C918115E1F081E08093240181E0A1
:1066D0002B96E2E10C94BD548135BCE79B0731F465
:1066E000FB018581811561F0C9DFF1CF82359C47BF
:1066F00039F4DB0115968C91811511F0CBDFE7CFD2
:1067000090917A0380917B03892B0E94FE0E182FB3
:1067100073DE181731F0F201608171810E94781BDD
:106720005C014EEEE42E45E0F42E812C912C212CC0
:1067300066246394712CD7016D917C91CC24CA940A
:10674000DD24DA9480E0282F30E0FB01E80FF11D12
:10675000E80FF11D408151814115510539F0A41612
:10676000B50609F096018F5F6901EDCF10E0BFEF2C
:10677000CB16DB0609F44CC0F701448110912401CB
:10678000411110E0D70115963C90159716969C91F3
:106790001697F2012581211509F4CDC0111509F4D0
:1067A000CAC0311017C0930102C0220F331FCA9410
:1067B000E2F76901922B16969C932091A5093091DE
:1067C000A6092233310530F462E370E07093A60924
:1067D0006093A509D30102C0AA0FBB1F8A95E2F7F7
:1067E000CD010197F70126812817190689F48091B8
:1067F000A7099091A809009709F44EC00E94004A89
:10680000C39708F449C081E0D70114968C9311E036
:10681000212ABFEF8B1A9B0AE7E0EE0EF11CF0E293
:106820008F16910409F087CFD20115968C918115AE
:1068300009F4E1C0211409F4DEC00E946F4A90936C
:10684000A8098093A7098091A409883008F591E0F0
:10685000980F9093A40999E0F201DE01119601903E
:106860000D929A95E1F7BDE08B9FC0011124845CE5
:10687000964F29E0FE013196DC0101900D922A9598
:10688000E1F72FEF3FEFFC0132872187B486A38623
:10689000822D809581701CCF00913A0930903B0980
:1068A000E0E0F0E0031113C0EE15FF0509F4B0CFEE
:1068B000802F90E0FC01EE0FFF1FEE5CF64F9182FF
:1068C000808201968370992780933B09A1CFC02EC7
:1068D000D12CF601EE0FFF1FEE5CF64F20813181C7
:1068E000B7E0B29FC001B39F900D1124FC01E251AB
:1068F000FA4FFB87EA87B701CF015CDEFC01009706
:10690000A9F021E024838E159F0509F481CF8091A1
:106910003A0908130BC06A857B85E617F70731F43F
:10692000C60101968370992780933A09C6010196A2
:10693000082F0370B7CF292F30E0311021C0D301C9
:1069400002C0AA0FBB1F8A95E2F7CD010197281755
:10695000390789F010E0F30102C0EE0FFF1FCA945F
:10696000E2F76F01C094D70116968C9116978C218F
:1069700016968C934DCF411571F3C4014FDDEACFCC
:10698000A9010C2C02C0559547950A94E2F7C9015C
:10699000019782239323892B59F540FF29C0F701E2
:1069A00082819381892B01F187E0FE013196DF011D
:1069B0001D928A95E9F70E946F4A9C018B839C8304
:1069C00084E08D83F70192818381792F988789876D
:1069D00009811A8144E05E816F810E940017D7010E
:1069E00015961C92132DB7CF60E0C401B9DCF7CF28
:1069F000142F1170B0CF90913A0980913B099817EC
:106A000011F0B5DD45CFADDC1092A8091092A709B1
:106A1000F4DC3ECF809125011F928F938091260157
:106A20001F928F93809129011F928F9380912A0149
:106A30001F928F9380912B011F928F9380912C0135
:106A40001F928F9380E09EE09F938F930E94AC0CE7
:106A50008DB79EB70E960FB6F8949EBF0FBE8DBF32
:106A60000895CF93C82F1F928F938AE99FE09F9339
:106A70008F930E94AC0C81E001C0880FCA95EAF7A1
:106A80000E946A130E9415130F900F900F900F90A1
:106A9000CF910895893209F46DC010F5833109F45E
:106AA00081C040F4873009F4DDC08B3051F18FE5AF
:106AB0009FE0ECC0843109F45DC092EE980F9A30EB
:106AC000B0F78D518093AD09843009F075C089E22B
:106AD00091E09093AC098093AB0986E292E091C07B
:106AE000803509F4D8C030F4883359F08F34F9F682
:106AF0008AE0D2C0813509F4E7C08235C1F681E071
:106B0000CBC084E89FE09F938F930E94AC0C82DF00
:106B10001F9281E08F931F9288E08F938DE79EE014
:106B20009F938F930E94AC0C8DB79EB708960FB6BB
:106B3000F8949EBF0FBE8DBF2091AD09211509F4B9
:106B4000CCC08091A9099091AA09009711F480E026
:106B500092E09F938F931F922F938DE49FE09F93DA
:106B60008F930E94AC0C0F900F900F900F900F908E
:106B70000F90089581E89FE09F938F930E94AC0C43
:106B80000F900F908091AD09811509F4AEC010925D
:106B9000AD091092AC091092AB091092AA0910929B
:106BA000A909CACF83E79FE09F938F930E94AC0C03
:106BB00031DF0F900F90C0CF68F48230C1F1833085
:106BC000C1F48AE291E09093AC098093AB0989E12A
:106BD00092E017C08530A1F18630D9F11092AD094D
:106BE00080E79FE09F938F930E94AC0C0F900F90D3
:106BF0000CC08CE291E09093AC098093AB0984E0E7
:106C000092E09093AA098093A9098091AD0981151A
:106C100009F492CF1F928F938CE69FE09F938F93FE
:106C20000E94AC0C0F900F900F900F9085CF8BE2CD
:106C300091E09093AC098093AB098DE092E0E1CFB5
:106C400086E291E09093AC098093AB0985E392E0F2
:106C5000D8CF85E291E09093AC098093AB0988E4AA
:106C600092E0CFCF81E080932C0184E180932B01CF
:106C70008AE080932A018EE18093290188E0809345
:106C8000260188E28093250182E69FE09F938F93FF
:106C90000E94AC0C8ECF86EFE091AB09F091AC096D
:106CA0003097C1F02081082E000C990B820F911DA6
:106CB000811521E0920754F497FD0AC080831F924A
:106CC0008F9389E59FE0AACF8FEFE6CF8FEFF6CFC6
:106CD00080E0F4CF86E59FE0D9CF89E49FE09F93E1
:106CE0008F930E94AC0C0F900F900895A4E0B0E039
:106CF000ECE7F6E30C94AA54EBEFE80FEF3308F05F
:106D000078C1F0E0EB5AF94A0C945C540E943519B2
:106D10001F921F921F928F938DE793E19F938F9302
:106D20000E94AC0CCE0104960E9433198C8183FB27
:106D3000882780F91F928F938C8182FB882780F9A6
:106D40001F928F938C81869581701F928F938C8177
:106D500081701F928F938C811F928F9384E393E1B4
:106D60009F938F930E94AC0CCE0101960E9439191B
:106D70008A8183FB882780F91F928F93898187FB03
:106D8000882780F91F928F93898186FB882780F955
:106D90001F928F93898185FB882780F91F928F939B
:106DA0008981829581701F928F93898183FB8827C7
:106DB00080F91F928F93898182FB882780F91F9227
:106DC0008F938A81869581701F928F938A818170BB
:106DD0001F928F938981869581701F928F938981ED
:106DE00081701F928F938A818F9389818F9385E31E
:106DF00092E19F938F930E94AC0C0FB6F894DEBF84
:106E00000FBECDBFCE0103960E943D198B818695A2
:106E1000869586951F928F938B8181701F928F9399
:106E20008B811F928F9382E092E19F938F930E94B8
:106E3000AC0C0FB6F894DEBF0FBECDBF81E0249638
:106E4000E9E00C94C6548EE394E19F938F930E94E3
:106E5000AC0C0E942A190F900F90F0CF8DE490E1B6
:106E60009F938F930E94AC0CF6CF80914604807F55
:106E70008093460486E290E19F938F930E94AC0C2E
:106E80008AE394E19F938F930E94AC0C81E08093FE
:106E9000AE090F900F900F900F90D0CF8EE194E13C
:106EA0009F938F930E94AC0C0F900F908091FE08DF
:106EB0009091FF08892B11F20E942A0EBFCF90916A
:106EC0004604892F8E7F90FF81608093460480FF67
:106ED00003C082E194E1C4CF85E094E19F938F9356
:106EE0000E94AC0C80914604817F80934604B3CF0E
:106EF00090914604892F8D7F91FF82608093460494
:106F000081FF0AC088EF93E19F938F930E94AC0C9E
:106F1000809146048160E9CF8AEE93E1A1CF909100
:106F20004604892F8B7F92FF84608093460482FF02
:106F300003C08BED93E1E8CF8BEC93E191CF90917F
:106F40004604892F877F93FF88608093460483FFE0
:106F500003C08FEB93E1D8CF82EB93E181CF8DE536
:106F600092E09F938F9383E290E19F938F930E948F
:106F7000AC0C8FCF0E947B4AE62ED72EC82EB92E9E
:106F8000F090F709F7FAFF24F0F80E94E049082F83
:106F90000E94C449182F0E94C647BF92CF92DF9229
:106FA000EF921F92FF921F920F931F921F931F92B7
:106FB0008F938FE99FE09F938F930E94AC0C39CF02
:106FC0000E9415139091F709892F97FB87F9805834
:106FD0008093F70987FF03C088EA93E141CF8DE9E9
:106FE00093E13ECF80E03DDD29CF8953FCCF8D5129
:106FF000FACF8BE993E19F938F930E94AC0C0F9093
:107000000F9080E01CCF80E0089580E00895CF933A
:10701000C82F8091AE09813091F0823009F448C0C8
:1070200081114AC00E94B917823209F047C08C2FE3
:10703000EADF811102C08C2F59DECF9108950E94A2
:10704000B9178232A1F38C2FE0DF811124C0C43143
:1070500021F168F4CB3079F0C03121F184E99FE06F
:107060009F938F930E94AC0C0F900F9018C0C93261
:10707000A1F0C83399F786E290E19F938F930E9425
:10708000AC0C86E99FE09F938F930E94AC0C0F900D
:107090000F900F900F9081E003C01092AE0980E036
:1070A0008170CBCF82E08093AE0988E3F3DCF3CF2D
:1070B0008C2FF0DC81E0C1CF1092AE0980E0BDCF13
:1070C000A1E0B0E0E6E6F8E30C94AF548E010F5F68
:1070D0001F4F21E030E040E050E0CCD28981219682
:1070E000E4E00C94CB5484E00895AAC10895D7C17C
:1070F000089582C3089595C30895A8C30895BBC396
:107100000895CEC30895E1C30895CF92DF92FF9210
:107110000F931F93CF93DF93CDB7DEB72A970FB6A8
:10712000F894DEBF0FBECDBFC090FE08D090FF0820
:1071300081E090E09093FF088093FE087FD100E00B
:1071400010E011C04F2D612F802F0E94FF0C9C0179
:107150004F2D612F802FA3D1F39483E1F812F2CF4A
:107160001F5F153011F0F12CEDCF0F5F043041F7A8
:107170001A8219821C821B821E821D8218861F821F
:1071800088EC90E09A878987F12C8E010F5F1F4F62
:10719000B8018F2DB0DFF394E0E2FE12F9CF8AE060
:1071A000F80111928A95E9F7F12CB8018F2DA7DF2C
:1071B000F394F0E2FF12F9CF86E0F80111928A957C
:1071C000E9F7F12CB8018F2D9EDFF394F0E2FF1266
:1071D000F9CFD092FF08C092FE082A960FB6F89415
:1071E000DEBF0FBECDBFDF91CF911F910F91FF90FA
:1071F000DF90CF9008950F931F938A019B0140E089
:1072000050E0BC0180E090E071D11F910F91089592
:107210000F931F938A019B0140E050E0BC0180E086
:1072200090E091D11F910F910895843028F465303A
:1072300018F4433108F404C180E090E0089580E13F
:10724000089513D2CB0108950F931F938A019B01D8
:1072500040E050E0BC0180E090E00CD21F910F9123
:1072600008950F931F938A019B0140E050E0BC01F9
:1072700080E090E043D21F910F910895E0D081C249
:10728000A4E0B0E0E6E4F9E30C94A254182F8031B6
:1072900008F0D0C0EAD1615071098109910910DF6D
:1072A0008111C8C0E2D14B015C01C12CD12C760107
:1072B000111140C034E0332E8E010F5F1F4FF801D3
:1072C000232D11922A95E9F7460157014FEF841AB1
:1072D000940AA40AB40AC701B601F2DE89838115B3
:1072E00009F4A8C0813009F0A0C02601370152E09E
:1072F000450E511C611C711CC501B401E1DE8A837D
:10730000811509F497C09FEF980F933028F5C301BA
:10731000B201D6DE8B83811519F0C8010E94D543D6
:107320004601570183E0880E911CA11CB11C750118
:107330006401C5CF8C149D04AE04BF0409F47AC067
:10734000C701B601BDDE2FEFC21AD20AE20AF20A65
:107350008111F0CF1150ACCF9BEF980F933090F587
:107360004601570193E0890E911CA11CB11CC30179
:10737000B201A6DE8B838115D1F2E4E0CE0ED11CE2
:10738000E11CF11CC501B4019BDE8C83811589F0E1
:107390008B819C818130FFEF9F0710F0982F882709
:1073A0002A81263049F0273051F0253011F40E940F
:1073B000712B46015701BBCF0E94E02AFACF0E94F1
:1073C000022BF7CF53014201843009F0B0CFC30143
:1073D000B20176DE782E4601570124E0820E911C20
:1073E000A11CB11CC701B6016D5F7F4F8F4F9F4F2E
:1073F00067DE7114F9F08115E9F08150990B4FEFB8
:10740000489F9001499F300D1124472D4150550B45
:10741000240F351F2150310908F489CF8FE99FE0EF
:107420000197F1F700C00000F5CF60E0C8010E94AD
:10743000C2437DCF2496E1E10C94BE540895089593
:107440000F931F93CF93DF93843030F5653020F591
:10745000433110F5C42FD0E0CC0FDD1F26E2629F30
:10746000C00DD11D11243EEB839FC00DD11D1124F1
:10747000CE0189960E94A655082F10E0102F0027F4
:10748000CE018A960E94A6559801282BC901DF914A
:10749000CF911F910F91089580E090E0F8CF1F9356
:1074A000CF93DF93962F122F632F8430D8F495302B
:1074B000C8F44331B8F4C42FD0E0CC0FDD1F26E26E
:1074C000929FC00DD11D11249EEB899FC00DD11D2F
:1074D0001124CE0189960E94C755612FCE018A964C
:1074E0000E94C755DF91CF911F910895A0E0B0E0B1
:1074F000ECE7FAE30C94A7546B017C01E801460128
:107500005701820E931EA41EB51EC814D904EA04A6
:10751000FB0429F4CDB7DEB7ECE00C94C35488EF3C
:10752000C81682E0D806E104F10458F4C601899631
:107530000E94A65589938FEFC81AD80AE80AF80A5C
:10754000E4CF80E0F7CFA0E0B0E0E9EAFAE30C9402
:10755000A1546B017C0149015A01E80128EFC216D0
:1075600022E0D206E104F10410F588EF92E0A0E0F9
:10757000B0E08C199D09AE09BF0988159905AA05C7
:10758000BB05A8F01B0139E2230E311C8091FE08D7
:107590009091FF08892B81F000E010E0C801A0E085
:1075A000B0E0081519051A041B0408F449C0CDB74A
:1075B000DEB7E2E10C94BD54340100E010E0C0FEFF
:1075C0000DC0CB0188960E94A655988189279827DF
:1075D000892781159C4789F101E010E0D701C60198
:1075E000880D991DAA1DBB1D80FF14C09401215058
:1075F000310939012E01420E531EC101880D991D1A
:107600000E94A655F201908181159C4719F48FEFD5
:10761000F2018083FE01E00FF11F2FEF0615170521
:1076200008F0BACF9081818181159C4711F42083A5
:1076300021830E5F1F4F3296F1CF8FEF8883CCCF1F
:107640008C0D9D1DAE1DBF1D883F9240A105B1054B
:1076500048F4FE01E00FF11F6081C101800F911F0E
:107660000E94C7550F5F1F4F99CF6FE979E080E007
:1076700090E008954F925F926F927F92AF92BF9287
:10768000CF92DF92EF92FF920F931F93CF93DF93EE
:107690006B017C0129013A0158018B010F59194FE7
:1076A000C0E0D0E0CE01A0E0B0E0C415D5051604DE
:1076B000170478F0DF91CF911F910F91FF90EF9019
:1076C000DF90CF90BF90AF907F906F905F904F9082
:1076D00008958C0D9D1DAE1DBF1D8F399940A105CC
:1076E000B10550F4C8018C0F9D1F0E94A655F501ED
:1076F00081935F012196D6CF80E0F9CF4F925F92C0
:107700006F927F92AF92BF92CF92DF92EF92FF92F1
:107710000F931F93CF93DF936B017C0129013A01F3
:1077200058018B010F59194FC0E0D0E0CE01A0E005
:10773000B0E0C415D5051604170478F0DF91CF9199
:107740001F910F91FF90EF90DF90CF90BF90AF907F
:107750007F906F905F904F9008958C0D9D1DAE1D92
:10776000BF1D8F399940A105B10548F4F501EC0F13
:10777000FD1F6081C8018C0F9D1F0E94C755219677
:10778000D5CFA0E1B0E0E7ECFBE30C94A354FE01FD
:10779000319680E1DF011D928A95E9F70AE910E050
:1077A0009FE9492E99E0592E612C712C21E6A22ED9
:1077B00026E0B22E4F0173016201B1E14B16510474
:1077C000610471041CF080E1C82ED12CA601B50122
:1077D000C4010E94B855AC0CBD1C0D2C000CEE0869
:1077E000FF084C185D086E087F080150104019F71B
:1077F0006096E0E10C94BF54282FCB01203270F446
:107800004AE0249F90011124B9016F5D7C4F4AE04A
:1078100050E00E94965580E090E008958FEF9FEF32
:107820000895282FCB01203270F44AE0249F900164
:107830001124B9016F5D7C4F4AE050E00E94E5558C
:1078400080E090E008958FEF9FEF0895282FCB01FF
:10785000203270F44AE0249F90011124B9016F593D
:107860007B4F4AE050E00E94965580E090E00895FA
:107870008FEF9FEF0895282FCB01203270F44AE05C
:10788000249F90011124B9016F597B4F4AE050E0C9
:107890000E94E55580E090E008958FEF9FEF0895F6
:1078A000282FCB01203270F446E0249F9001112450
:1078B000B9016F557A4F46E050E00E94965580E03E
:1078C00090E008958FEF9FEF0895282FCB0120328D
:1078D00070F446E0249F90011124B9016F557A4F4E
:1078E00046E050E00E94E55580E090E008958FEF7B
:1078F0009FEF0895CF93DF93EB0186319C4719F5F5
:107900000E94B9179D819115A1F08A7A91E08111A9
:1079100001C090E09093AF09811549F085E30E9482
:1079200016490E949E1880E0DF91CF91089589E268
:10793000F6CF8091AF09811521F085E30E942D4992
:10794000F0CF89E2FBCF81E0EFCF0F931F93CF936E
:10795000DF93EC018B016CD08091B00990917A0398
:10796000292F30E02095309550E028233523232B14
:1079700021F089238093B0096FD0CB372CE7D20751
:1079800059F4F8018581811529F080917A030E94CC
:10799000FE0E64D080E011C0C034F2E5DF0750F580
:1079A000C03222E5D20758F5C11580E5D80750F45A
:1079B000C115E0E4DE0778F581E0DF91CF911F91FA
:1079C0000F910895CE01905581159240A8F785E05A
:1079D000D695C7958A95E1F7CF708C2F2AD081155F
:1079E00059F3F8018581811114C00E94CA170E94C1
:1079F0009E18D0CFCE01805C92458097E8F6CF717B
:107A00008C2F17D08115C1F2F8018581811509F4F9
:107A1000C1CF8C2FBECFF8018681803168F6858179
:107A20008111CACF8D2F8F7004D091E08927C5CFE7
:107A300008952091B00930E041E050E002C0440FC9
:107A4000551F8A95E2F72423352381E0232B09F47F
:107A500080E0089581E00895FDCF08950F931F936E
:107A6000CF93C82F01E010E001C0000F8A95EAF71C
:107A70008091B0098023811113C00E9493178C1349
:107A800002C00E94C5188C2F0E948C138091B009EF
:107A900080278093B009E0DFCF911F910F91089567
:107AA0008C2F0E949613F2CF0895CF93DF93EC01B1
:107AB000FB018581811509F4CBC09E01305723322B
:107AC000310508F0ABC087EF99E00E943919FE013B
:107AD000E150F047E232F10520F4EC56F94A0C94FB
:107AE0005C548091F70981608093F70990C0809180
:107AF000F80988608093F8098AC08091F70982604C
:107B0000F3CF8091F7098460EFCF8091F709886007
:107B1000EBCF8091F8098160EDCF8091F809826008
:107B2000E9CF8091F7098061DFCF8091F70980620A
:107B3000DBCF8091F7098064D7CF0E941513809125
:107B4000F7098068D1CF8091F7098C60CDCF809103
:107B5000F8098360CFCF8091F7098E7FC5CF8091E0
:107B6000F809877FC7CF8091F7098D7FBDCF8091BE
:107B7000F7098B7FB9CF8091F709877FB5CF8091C7
:107B8000F8098E7FB7CF8091F8098D7FB3CF8091B0
:107B9000F7098F7EA9CF8091F7098F7DA5CF8091BE
:107BA000F7098F7BA1CF0E9415138091F7098F777A
:107BB0009BCF8091F709837F97CF8091F8098C7FC5
:107BC00099CF8091F709992782FF939590FB82F9CD
:107BD00090FB83F989CF8091F809982F909590FBBD
:107BE00080F990FB81F986CF9091F709892F8F7BDF
:107BF00096FF806479CF0E9415139091F709892F21
:107C000097FB87F9805870CF81E00E94451987EF74
:107C100099E00E943B190E94151380E0DF91CF91FB
:107C2000089580E0F2CF9091F709892F8F7E94FF1D
:107C300080615ACF9091F709892F8E7F90FF8160E4
:107C400053CF9091F809892F877F93FF886052CF97
:107C500081E0E4CF282F35EB2303C001112497FFE7
:107C600004C080589109892F089580589F4FFBCFF9
:107C70008091B70980FF0DC060912A0170E0660F06
:107C8000771F60387105B0F561157105A9F1862F70
:107C9000089581FF07C060912A0184E0689FB001C8
:107CA0001124EFCF82FF04C060912A0188E0F6CF53
:107CB0009091B6099115D9F02091290180912A015E
:107CC000682F70E0921730F043E0660F771F4A95F7
:107CD000E1F7D7CF899FC001112433E0880F991FA6
:107CE0003A95E1F7622F70E00E942754CACF68E00E
:107CF00070E0CDCF8FE7089581E008958091B709B6
:107D000080FF0CC06091260170E0759567957595B0
:107D100067956115710549F1862F089581FF06C0A9
:107D20006091260170E075956795F3CF609126010B
:107D300082FD0BC09091B5099115A1F060912501CC
:107D400080912601961738F0682F70E06038710531
:107D500000F38FE70895899FC001112470E00E940D
:107D60002754F4CF61E070E0D7CF81E00895E3E3DA
:107D7000E80FE331A0F5F0E0EA54F94A0C945C54C2
:107D800077DF81958093BB09089572DFFBCF70DFA9
:107D900081958093BA0908956BDFFBCFAFDF8093A5
:107DA000BC090895ABDF8195FACFA8DF8195809358
:107DB000BD090895A3DFFBCF815D990B21E030E081
:107DC00001C0220F8A95EAF78091B909822B80932E
:107DD000B90908958091B70981608093B709089522
:107DE0008091B7098260F9CF8091B7098460F5CF9F
:107DF0004091BA098D3C59F48091BB0987FF0DC0B1
:107E00001092BB09411559F41092B60908C08E3C76
:107E100081F48091BB0918169CF3411581F0809183
:107E2000BC099091BD09892B811159C01092B509E7
:107E300008958F3C41F447FFF0CF1092BA0980912A
:107E4000BB098115E0CF803D19F41416B4F3E5CFDA
:107E50009091BC09893D29F41916FCF61092BC09D1
:107E6000DCCF8A3D19F497FFD8CFF8CF9091BD09A8
:107E70008B3D29F497FFD1CF1092BD09CECF8C3D19
:107E800019F41916CCF3C9CF9FE2980F983090F4EB
:107E9000815D990B21E030E0B90102C0660F771FC8
:107EA0008A95E2F7CB0180959091B9098923809357
:107EB000B909B3CF8D3D31F48091B7098E7F80939E
:107EC000B709ABCF8E3D21F48091B7098D7FF7CFF5
:107ED0008F3D09F0A2CF8091B7098B7FF0CF089535
:107EE0008091460483FF96C086E794E19F938F9329
:107EF0000E94AC0C8091B9091F928F9381E794E1A5
:107F00009F938F930E94AC0C8FE694E19F938F9385
:107F10000E94AC0C8091BA09282F082E000C330B5C
:107F20003F938F938CE694E19F938F930E94AC0CC8
:107F30008AE694E19F938F930E94AC0C8091BB09D9
:107F4000282F082E000C330B3F938F9387E694E184
:107F50009F938F930E94AC0C85E694E19F938F933F
:107F60000E94AC0C8091BC09282F082E000C330B0A
:107F70003F938F9382E694E19F938F930E94AC0C82
:107F800080E694E19F938F930E94AC0C8091BD0991
:107F9000282F082E000C330B3F938F938DE594E12F
:107FA0009F938F930E94AC0C8AE594E19F938F93EB
:107FB0000E94AC0C8DB79EB780960FB6F8949EBF0A
:107FC0000FBE8DBF8091B6091F928F9387E594E114
:107FD0009F938F930E94AC0C85E594E19F938F93C0
:107FE0000E94AC0C8091B7091F928F9382E594E1B7
:107FF0009F938F930E94AC0C8FE494E19F938F9397
:108000000E94AC0C8DB79EB70C960FB6F8949EBF2D
:108010000FBE8DBF0E946F4A2091BA093091BB09F3
:10802000232B211521F08093B3099093B40920915B
:10803000BC093091BD09232B211521F08093B10992
:108040009093B20988EB99E0D2C786E0E8EBF9E0BB
:10805000DF011D928A95E9F71092B6091092B509D1
:108060001092B7090895FC01828181110DC08381AE
:1080700081110AC08481811107C081E0958191112D
:1080800001C080E08170089581E0FCCFA6E0B0E0FF
:10809000ECE4F0E40C94AE5486E0E8EBF9E09E01E9
:1080A0002F5F3F4FD90101900D928A95E1F7109211
:1080B000BA091092BB091092BC091092BD098B81BC
:1080C0009C81892B8901811589F08091B309909158
:1080D000B4090E94004A9C018091B6098115A9F15A
:1080E00090912B019217130608F43CC08D819E815C
:1080F000892B811591F08091B1099091B2090E946C
:10810000004A9C018091B509811509F459C09091EC
:1081100027019217130608F461C0B80188EB99E0B3
:108120000E945D49811104C088EB99E09CDF8111B8
:10813000D7DE86E0F801A8EBB9E001900D928A95B0
:10814000E1F72696E5E00C94CA5440912C019AE0A0
:10815000499FA00111244217530740F68F5F809377
:10816000B60902C08F3FD1F7FB80F11451F080DDDA
:1081700091E01F140CF09FEF899F802D11248093B4
:10818000BA09FC80F11451F073DD91E01F140CF07A
:108190009FEF899F802D11248093BB098091BA099C
:1081A000811509F4A3CFF090BB09F11409F49ECF17
:1081B00051DD8093BA098F2D4DDD8093BB0996CF99
:1081C000409128019AE0499FA001112442175307CA
:1081D00008F0A3CF8F5F8093B50902C08F3FD1F71E
:1081E000FD80F11451F08ADD91E01F140CF09FEF37
:1081F000899F802D11248093BC09FE80F11451F0D9
:108200007DDD91E01F140CF09FEF899F802D1124DC
:108210008093BD098091BC09811509F47ECFF0904F
:10822000BD09F11409F479CF15DD8093BC098F2DB8
:1082300011DD8093BD0971CF81E00895A1E0B0E028
:10824000E4E2F1E40C94AC548C017B01AAD08111DE
:1082500034C0F7018581811581F10E94B917D82EAC
:108260000E94CD17D82AD9820E94E4179981982BB1
:1082700099830115F0E51F0728F5011580E218071D
:1082800098F50115E7E01E07C1F098F4C801805E7B
:108290009109089790F0AE014F5F5F4FB701C80199
:1082A000CBDF811551F0B701C8016BD0898166D051
:1082B00004C001158FE0180771F781E02196E7E00F
:1082C0000C94C854003EE2E51E0748F40036F2E57F
:1082D0001F0798F7C801925580349105DBCFC8017C
:1082E00087579C470597D6CFF70186818031D2CF3B
:1082F0000F931F93CF93DF938C01D62FC72F51D0AD
:10830000811114C009378CE7180749F48D2F9C2F71
:108310004BD080E0DF91CF911F910F9108950A37E4
:108320001C4721F48D2F9C2FD1D0F3CF81E0F2CFC9
:108330009091D30989029001112437FF03C08093E3
:10834000D30908952F3731051CF4980F9093D30962
:1083500008959C0180E090E0F901E80FF91FE49195
:10836000E41307C091E08927F901E80FF11D84911A
:1083700008950196861780F380E008958093D409CC
:1083800008959C01FB0199E0A5EDB9E001900D92E3
:108390009A95E1F73093DD092093DC091092D30917
:1083A00008958091D2090895CF93DF93EC018091D5
:1083B000D209811135C08091DC099091DD09892BAA
:1083C00079F18D81811599F081E0B2DF8091D40936
:1083D0000E94FA1289E0E5EDF9E0A9ECB9E001901C
:1083E0000D928A95E1F78091D3098093C80986E0C0
:1083F000FE01A9ECB9E001900D928A95E1F7809118
:10840000C8098093D20989EC99E00E94DC1210928D
:10841000D2098D81811104C08091D4090E94FF127C
:10842000DF91CF9108950F931F93CF93DF93C09166
:10843000DC09D091DD090091D409602FCE010E94A2
:108440008C2C81309105B1F5802F82958F70802B17
:108450008F7011E0003108F410E01295107F182B96
:10846000C11520E2D207F8F4C11581E0D80738F52C
:108470000C2F812F8D704C2F811521F16AE08FEB2D
:1084800094E167DF282F30E02115310549F4402FB2
:108490006EE189E994E15DDF282F30E0811541F03C
:1084A000C901912B07C0CE0190528115904340F035
:1084B00080E090E0DF91CF911F910F9108951D2BE7
:1084C000DD27D6CF68E087EB94E1DBCFCF93DF9356
:1084D000EC018091D209811130C08D81811561F04C
:1084E000A2DF27E0EFEBF9E0DF011D922A95E9F723
:1084F0009093C7098093C6098091C6099091C709D6
:10850000892BD9F08D81811531F08FEF11DF8091AA
:10851000D3098093BE0986E0FE01AFEBB9E001907C
:108520000D928A95E1F78091BE098093D2098FEB75
:1085300099E00E94DC121092D209DF91CF91089548
:10854000FC01A081B1818D91B183A0830895A0E049
:10855000B0E0EDEAF2E40C94AA54E82FF0E0E7531F
:10856000FB4EB490282F26952695269530E0F901EC
:10857000E759FA4E0491877010E0082E02C0159555
:1085800007950A94E2F701701127F901E75AFA4EAC
:10859000E490F12C082E02C0F594E7940A94E2F7D7
:1085A000E0FAEE24FF24E0F8F901E75BFA4EC4910B
:1085B000D0E002C0D595C7958A95E2F7C170DD2756
:1085C000C62ED12C0115110549F5E114F10431F045
:1085D00086EE0E94DF0FC601009771F5B6018B2D64
:1085E0000E94C410C601009779F5E114F104A1F5C9
:1085F0000115110531F081EE0E946F10C601009740
:10860000C9F5CD2B31F08CE20E94DA10C114D104EF
:10861000C9F5CDB7DEB7E9E00C94C65481EE0E94EF
:10862000DF0FC601009789F2EFE9FFE03197F1F71C
:1086300000C000000197F6CFEFE9FFE03197F1F7B6
:1086400000C000000197C8CFEFE9FFE03197F1F7D4
:1086500000C000000197C7CF86EE0E946F10C601D0
:10866000009731F2EFE9FFE03197F1F700C0000029
:108670000197F6CFEFE9FFE03197F1F700C0000076
:108680000197BDCF8FE99FE00197F1F700C000008F
:1086900091E0C91AD108BACFA0E0B0E0E2E5F3E476
:1086A0000C94AA548C01D62FF72EE42E8D2F9F2DDB
:1086B000F80109958115B9F0813009F060C08D2F5E
:1086C0009F2DF8010995C82F813091F48D2F9F2D92
:1086D000F80109950E94DA108E2D90E0009709F0BC
:1086E00046C0C111E3CFCDB7DEB7E9E00C94C65464
:1086F000823039F48D2F9F2DF80109950E94DF0FEC
:10870000EBCF833039F48D2F9F2DF80109950E940E
:108710006F10E2CF843001F78D2F9F2DF80109955E
:10872000C82FC12CD12C8AE0B82E2C2F2053330B0C
:10873000C9012A30310568F0C114D10469F28FE90A
:108740009FE00197F1F700C0000091E0C91AD1083D
:10875000F3CFBC9C9001BD9C300D11246C01C20E66
:10876000D31E8D2F9F2DF8010995C82FDECFEFE97D
:10877000FFE03197F1F700C000000197AFCF6E2DF9
:10878000E6DE94CFA2E0B0E0E8ECF3E40C94B15460
:10879000462F9A838983BE016F5F7F4F80EA92E400
:1087A0007BDF2296E2E00C94CD5460E0EBCFA0E0BA
:1087B000B0E0EDEDF3E40C94A9547C015B01C42F0F
:1087C000D22FFC0185818115C1F04093E00987D645
:1087D0009093DF098093DE0980E28C0F883040F4AB
:1087E000C77081E001C0880FCA95EAF70E94E110C6
:1087F000CDB7DEB7EAE00C94C5541091E00914132C
:1088000038C08091DE099091DF09FAD56C01B7017B
:10881000C5010E94112CC816D90658F5C0E2CD0F2B
:108820001D17C9F080E2810F883048F4177081E08D
:10883000012E01C0880F0A94EAF70E94E610C830A2
:1088400050F491E08D2F877001C0990F8A95EAF757
:10885000892F0E94E110802F0E94DA10C83040F664
:10886000D77081E001C0880FDA95EAF70E94E61020
:10887000BFCF80E28C0F883008F0BACFC77081E09C
:1088800001C0880FCA95EAF7F1CF0F93FC01CB0125
:10889000E851FC47E730F10588F5E753F94A0C94B5
:1088A0005C5406E221EE41EE6AE17CE780DF80E085
:1088B0000F91089507E225EE45EE6BE17CE7F6CFD8
:1088C00006E221EE40EE68E17CE7F0CF07E225EE1C
:1088D00044EE69E17CE7EACF06E221EE42EE6CE18C
:1088E0007CE7E4CF07E225EE46EE6DE17CE7DECFE4
:1088F00008E221E045EE6EE17CE7D8CFFB018581FF
:1089000081111092E00981E0D3CFFA01309709F08C
:1089100009950895CF93DF93EC014A855B856E85B9
:108920007F85F3DF8B810E94D6178C810E94C2174E
:108930000E949E1886E0FE0111928A95E9F7DF9168
:10894000CF910895CF93DF93EC018D8181FD10C00D
:1089500082608D838B810E94D0178C810E94BC170E
:108960000E949E18488559856E857F85CE01CDDF92
:108970001092E4091092E3098D8180FD02C0CE01BE
:10898000C9DFDF91CF9108950F931F93CF938C018F
:10899000FB01C581C115B1F08091E3099091E40913
:1089A0000097A9F08017910791F099270E94302C29
:1089B000FC0185818460858311830083CF01C2DF40
:1089C0000E94E1178C2FCF911F910F910895C0E065
:1089D000F9CFEF92FF920F931F93CF93DF938C0108
:1089E0007B0197558115914030F081E0CDB7DEB71E
:1089F000E6E00C94C954E801DD270E942D2CC8172D
:108A0000D90708F047C0CE010E94302CEC01F701D5
:108A100085819D8180FB90F99D83811519F15FD53A
:108A20009093E2098093E1098A818F5F8A830E9493
:108A3000B9178B830E94CD179B81982B9B830E9433
:108A4000E4178C834E815F816E857F85CE015DDF6B
:108A50008D8181FF02C000E010E01093E4090093D3
:108A6000E309C3CF4C855D856E857F85CE014DDFE3
:108A70008D8181FFBACFCE014DDF8091E3099091C6
:108A8000E4098017910709F0B0CF1092E409109221
:108A9000E309ABCF80E0AACFA9E0B0E0E2E5F5E4DE
:108AA0000C94AF548091E3099091E409892B21F152
:108AB0008091E1099091E209A3D48C01BE016F5F1E
:108AC0007F4F89E0FB0111928A95E9F78091E309D4
:108AD0009091E4090E94112C8017910768F480910D
:108AE000E3099091E40999270E94302CFC018581CB
:108AF00082FD02C0CF0126DF2996E4E00C94CB541E
:108B0000CF93DF939C01FB0127378CE7380739F0BF
:108B100028373C47C9F081E0DF91CF9108958581E6
:108B2000811571F018D00E948C131BD0D82F16D04D
:108B3000C82F11D04D2F6C2F0E94A61480E0ECCFCF
:108B40000AD00E949613F1CF8581811511F006D0CD
:108B5000EACF04D0F6CF80912F01089580912E01A5
:108B6000089580912D01089585E290E00E94A65518
:108B70008A3989F486E290E00E94A6558D3859F42E
:108B800087E290E00E94A65591E08A3309F090E0D8
:108B9000892F8170089580E0FCCFCF93C82F6AE9B8
:108BA000811101C06FEF85E290E00E94C7556DE82A
:108BB000C11101C06FEF86E290E00E94C7556AE3E1
:108BC000C11101C06FEF87E290E00E94C755CF91BD
:108BD0000895089588E290E00E94A655682F70E0FD
:108BE00080E090E008950895CF93C62FFCDF6C2FAE
:108BF00088E290E00E94C755CF91089580E0CDDFD4
:108C000060E070E0CB01F0DF0E9485380E943E39C1
:108C100081E0C3CFDEDFDEDFE6DFA6DF811101C04A
:108C2000EDCF08959C01FB018581811551F0A901CB
:108C300057574038510530F4822F0E94403980E068
:108C4000089581E008952FEFFC0120830895CF93CC
:108C5000DF93EC018881893029F08A3059F0DF9167
:108C6000CF9108950E94D82525E5829FC001112447
:108C70008983F5CF0E94FE25FBCFFC0180818930DE
:108C800019F08A3079F00895218130E0C901880F08
:108C9000991F820F931F6FEF70E00E941354862F6D
:108CA0000C94AD268181811102C00C94EB250C94AB
:108CB000DE25CF93DF93EC0188818238C1F038F450
:108CC000803871F0813881F0DF91CF910895833839
:108CD000D9F70E948C2089830E948F208A83F4CF49
:108CE0000E9492208983F0CF0E945F20FBCF0E94D8
:108CF0008620F8CFCF93DF93EC018881823839F159
:108D000038F4803869F08138B1F0DF91CF9108955F
:108D10008338D9F70E949220482F6A81898108C040
:108D2000D9810E948F20C82F0E948C204D2F6C2F3C
:108D30000E94E421EACF89810E94F3248981811174
:108D400003C00E947624E1CF0E941925DECF8981DD
:108D50000E948920DACFEF92FF920F931F93CF9357
:108D6000DF93EC01162FE8818091FC089091FD08BB
:108D7000892B69F0EE3F21F58981833018F0855009
:108D80008330F0F4612FCE010E94342919C07E0196
:108D90002FEFE21AF20AE43150F4E11551F0E150FC
:108DA000E33138F4F0E0E053F94A0C945C54EE3FC0
:108DB00049F3612FCE0147DF03C0198289E08A831E
:108DC000612FCE010E943F28CDB7DEB7E6E00C94BC
:108DD000C9548981823061F0833081F0813049F754
:108DE0008AD30E9475546A837B838C839D83E8CFEA
:108DF000F1DE1A821B821C826D83E2CF8091FE0815
:108E00009091FF08892BE1F27E0100E0802F0E9403
:108E1000891DF7018283738364830F5FF3E0EF0E94
:108E2000F11C053099F7CCCF8981823009F0C1CF90
:108E30006A817B818C819D810E947554D5DEC0CF73
:108E40004B816A8189810E947538982789279827E4
:108E50009D838C83B5CF2C813D81322723273227F8
:108E60004B816A8189810E947738AACF0E94853818
:108E7000A7CFC70102DFC7013DDFA2CFC701E7DEF1
:108E8000C70117DF9DCF0E94CD250E94502098CFAB
:108E90000E941F39898394CF0E94213998278927FE
:108EA00098279A8389838CCF8B81682F70E08D31CE
:108EB00008F086CF89819A81AE014C5F5F4F982779
:108EC000892798270E9424397BCF8091FE089091B2
:108ED000FF08892B09F474CF8B81682F70E08D31E6
:108EE00008F06ECF89819A81AE014C5F5F4F982761
:108EF000892798270E94313963CF0E943E3960CF7D
:108F00000E947338C7CF8B81682F70E08D3108F0D5
:108F100057CF89819A81AE014C5F5F4F982789278F
:108F200098270E94FB384CCF8B81682F70E08D31E1
:108F300008F046CF89819A81AE014C5F5F4F982738
:108F4000892798270E9408393BCF8091FE0890918D
:108F5000FF08892B09F434CFCE010E943F282FEF60
:108F600081EE94E0215080409040E1F700C0000085
:108F7000F2D226CF9093EA098093E909089504D2AA
:108F8000982F81E0913009F080E00895E091E9099F
:108F9000F091EA09309739F00190F081E02D309797
:108FA00011F00995089580E00895F0CF0895E091BB
:108FB000E909F091EA09309731F00280F381E02D60
:108FC000309709F009950895DC01E091E909F091E5
:108FD000EA09309759F084819581892B39F086E030
:108FE0008C930480F581E02DCD0109950895DC0175
:108FF000E091E909F091EA09309759F0868197816B
:10900000892B39F082E08C930680F781E02DCD0129
:1090100009950895A3E0B0E0E0E1F8E40C94B154C0
:109020009C018091E7099091E80982179307B1F0BC
:109030003093E8092093E709E091E909F091EA0902
:10904000309761F00084F185E02D309739F083E0AE
:1090500089833B832A83CE01019609952396E2E01A
:109060000C94CD54A3E0B0E0E8E3F8E40C94B154E0
:109070009C018091E5099091E60982179307B1F070
:109080003093E6092093E509E091E909F091EA09B6
:10909000309761F00084F185E02D309739F084E05D
:1090A00089833B832A83CE01019609952396E2E0CA
:1090B0000C94CD54E091E909F091EA09309731F030
:1090C0000284F385E02D309709F009950895CF9338
:1090D000DF93C0910601D0910701229650DF8115E0
:1090E00081F08091F70987FF0CC0C0910401D091F5
:1090F000050122969EE180E0915028F4DF91CF9106
:10910000089596E0F8CF29912115B1F38F5FF4CF40
:10911000CF93C82F811102C080E030C030DF8115AD
:1091200021F08091F70987FD0EC080910601909192
:109130000701FC013296089621912C1709F1E817D6
:10914000F907D1F7E9CF8C2F869586958695C03F94
:1091500018F7E0910401F0910501E80FF11D22815B
:1091600030E0C77081E090E002C0880F991FCA9577
:10917000E2F72823392381E0232B71F2CF91089560
:1091800081E0FCCF9C01FC0132968FEF90E0419191
:10919000461751F08F3F19F4411101C0892F9F5F8D
:1091A0009630A9F78F3F09F40895280F311D87FDE8
:1091B0003A95F901628308959C01FC013296285F7B
:1091C0003F4F8191861302C0DF011E92E217F30721
:1091D000C1F70895FC01862F869586958695603F98
:1091E00060F4E80FF11D677021E030E001C0220F4C
:1091F0006A95EAF78281822B82830895FC01862F8B
:10920000869586958695603F80F4E80FF11D67701E
:1092100081E090E09C0102C0220F331F6A95E2F7C3
:10922000B90160958281682362830895CF93C82F26
:10923000A6DE6C2F811559F08091F70987FF07C0D2
:109240008091040190910501C5DFCF91089580912F
:1092500006019091070196DFF8CFCF93C82F8FDEDC
:109260006C2F811559F08091F70987FF07C0809115
:10927000040190910501C2DFCF910895809106010C
:109280009091070199DFF8CF7ADE811579F080910E
:10929000F70987FF0BC0E0910401F09105013296B8
:1092A0008EE1DF011D928A95E9F70895E0910601AC
:1092B000F0910701329686E0F4CFDC01FB011196B4
:1092C0009C9111978181981322C012968C911297CC
:1092D000811519F0928189131AC013968C911397F6
:1092E000811519F09381891312C015968C911597E9
:1092F000811519F0958189130AC014969C919115D6
:1093000021F081E02481291303C080E001C081E0C5
:10931000817008950895FECF08958F5F8093330183
:10932000609130017091310180913201909133014F
:10933000F2CF83E08093330160913001709131016D
:109340008091320190913301E6CFE7CF089581E01B
:10935000809333016091300170913101809132012D
:1093600090913301D8CFF3CF089591E0811101C0DE
:1093700090E09093320160913001709131018091C1
:10938000320190913301C7CF8091320108958093CB
:1093900031016091300170913101809132019091E1
:1093A0003301B9CF809131010895809330016091EC
:1093B0003001709131018091320190913301ABCF36
:1093C00080913001089508950895FECF089508957D
:1093D0000895F9CF0895CF93FADF0E94B11EF8DF08
:1093E000C0E08C2F0E94891D672B682B692B31F4FC
:1093F000CF5FC530B1F780E0CF91089581E0FCCF19
:10940000CF93DF93EC016BD08C1B9D0BDF91CF9141
:10941000089585B7806885BF85B7806885BF089542
:109420001F921FB61F9211248F939F93AF93BF93E8
:109430008091EB09811113C08091CC0D9091CD0DDD
:10944000A091CE0DB091CF0D4196A11DB11D80937D
:10945000CC0D9093CD0DA093CE0DB093CF0DBF91B9
:10946000AF919F918F911F901FBE1F901895809173
:10947000D40D843031F10E94EC0E1092EB0988E19A
:1094800090E020E40FB6F894A895809360000FBE9A
:109490002093600083B7817F846083BF83B781603E
:1094A00083BF7894889583B78E7F83BF0FB6F89477
:1094B000A8958091600088618093600010926000A0
:1094C0000FBE08950E9415130C94F50E82E084BD22
:1094D00093E095BD9AEF97BD80936E0008952FB7E6
:1094E000F8948091CC0D9091CD0DA091CE0DB091BE
:1094F000CF0D2FBF08952FB7F8946091CC0D7091C8
:10950000CD0D8091CE0D9091CF0D2FBF0895789401
:109510001F921FB61F9211248F939F93AF93BF93F7
:109520008091CC0D9091CD0DA091CE0DB091CF0D2D
:109530000196A11DB11D8093CC0D9093CD0DA093EC
:10954000CE0DB093CF0DBF91AF919F918F911F9092
:109550001FBE1F90189581E08093E00080E2809309
:10956000D8001092C9008FE19EE40197F1F700C086
:10957000000087E090EBDC018093DD0D9093DE0D21
:10958000A093DF0DB093E00D88E19CE00FB6F89456
:10959000A895809360000FBE90936000FFCF88E194
:1095A0009CE00FB6F894A895809360000FBE90934E
:1095B0006000FFCFFF920F931F93CF93DF93182F7D
:1095C000EB011092BC0084EA8093BC0088DF082F76
:1095D000F92E8091BC0087FF27C08091B900887F59
:1095E000883029F08091B900887F803189F5109307
:1095F000BB0084E88093BC0072DF182F092F809194
:10960000BC0087FF1EC02091B900287F80E090E059
:10961000283191F081E090E0203411F480E090E076
:1096200091958195910908C0802F9F2DE9DEC8177B
:10963000D90778F68EEF9FEFCDB7DEB7E5E00C9453
:10964000CA54812F902FDCDEC817D907C0F6F2CF9D
:109650008FEF9FEFF1CF1092B9008CE08093B800AC
:1096600008950F931F93CF93DF93EB018093BB007B
:1096700084E88093BC0033DF182F092F8091BC0051
:1096800087FF11C02091B900287F81E090E0283247
:1096900011F480E090E0919581959109DF91CF914F
:1096A0001F910F910895CF3FDC0741F3812F902F39
:1096B000A7DEC817D90710F78EEF9FEFEFCFA0E016
:1096C000B0E0E5E6FBE40C94A654782EB62EA72E67
:1096D0006A01890104DF4C010431110518F10F3FC3
:1096E000100721F1C80164E170E00E941354F62EC6
:1096F000E72E6F2D7E2D872D5DDFEC01892BC9F4C0
:10970000EB2CFA2CCE0CDF1CEC14FD0411F020978E
:10971000C9F084E98093BC00CE01CDB7DEB7EDE09F
:109720000C94C254FF24F394E12CE3CF85E0F82E8F
:10973000FBCF0F3F1007E9F2C40162DE08171907DB
:10974000C0F6DECFB801F70181917F018ADFEC011D
:10975000DBCFA0E0B0E0EFEAFBE40C94A654782E57
:10976000B62EA72E6A018901BADE4C01043111051B
:1097700018F10F3F100721F1C80164E170E00E9469
:109780001354F62EE72E6F2D7E2D872D13DFEC015F
:10979000892BC9F4EB2CFA2CCE0CDF1CEC14FD0445
:1097A00011F02097C9F084E98093BC00CE01CDB7B9
:1097B000DEB7EDE00C94C254FF24F394E12CE3CF28
:1097C00085E0F82EFBCF0F3F1007E9F2C40118DE49
:1097D00008171907C0F6DECFF7018491B80141DF01
:1097E000EC01FFEFEF1AFF0AD9CFA0E0B0E0EBEFFA
:1097F000FBE40C94A554682E962E5A016901780159
:109800006EDE782E892E0431110520F10F3F1007EE
:1098100021F1C80164E170E00E941354162F072F54
:10982000612F702F862DC6DEEC01892BC1F0FFEF72
:10983000EF16FF06A9F3872D982DE2DDE816F9064D
:1098400078F784E98093BC00CE01CDB7DEB7EEE0B7
:109850000C94C15411E000E0E3CF15E0FCCFB70158
:10986000892DFFDEEC018501CA0CDB1C0C151D05E2
:1098700041F3209731F7B701F80181918F01F1DEB3
:10988000EC01F4CF282FCB01BA013091D40D343044
:10989000D1F42F702093E9002FEF3091E80035FDCF
:1098A00006C035ED3A95F1F700002A95B1F7209101
:1098B000E80025FF08C040E050E0CFD28091E800EA
:1098C0008E778093E8000895792F603229F440E282
:1098D00050E0682F82E0D6CF0895BC0143E050E00D
:1098E00084E0D0CFBC0146E050E084E0CBCFBC01A7
:1098F00040E250E084E0C6CFCF93DF93D82FC92F4A
:1099000043DD48E050E06D2F7C2F81E0BBDF88E035
:10991000ED2FFC2FAFEEB9E001900D928A95E1F7A3
:10992000DF91CF910895A0E2B0E0E9E9FCE40C9466
:10993000B1548091D40D8430F9F483E08093E90030
:109940008091E80082FF18C08091E80090E085FFD8
:1099500008C040E050E060E270E0CE010196CAD25B
:1099600091E08091E8008B778093E800911521F0D9
:1099700060E2CE010196EFD9A096E2E00C94CD54BE
:10998000089589E895E19F938F930E94AC0C809194
:10999000D30D0F900F90811107C032D48ED48091D7
:1099A000E20084608093E200089585E895E19F934A
:1099B0008F930E94AC0C1092D30D0F900F900895CE
:1099C00081E895E19F938F930E94AC0CC0DC81E00D
:1099D000CCDC0F900F9008958DE795E19F938F93C6
:1099E0000E94AC0C6091D00D81E0611101C080E05B
:1099F000A0DC0F900F90089589E795E19F938F93D6
:109A00000E94AC0C9091D40D81E0943009F080E07C
:109A10006091D00D9ADC0F900F9008952091ED0980
:109A20002F5F822F62E3E6D6911519F02093ED099E
:109A300008951092ED098091EE098115E9F0809169
:109A4000D40D8430B9F49091E9008091EC009F70BE
:109A5000879588278795892B95E09093E9009091C9
:109A6000EB0090FF04C09091EE0097FD08C08F704E
:109A70008093E9001092EE0908951092F100909100
:109A8000E80095FDFACF9091E80090FFF0CF90911B
:109A9000E8009E779093E800EACF42E061EC81E035
:109AA0002BD342E261EC84E027D342E261EC82E016
:109AB00023D342E260EC83E01FD342E261EC85E015
:109AC0001BD39091D40D81E0943009F080E0609137
:109AD000D00D23CC8091D60D893081F148F48230AD
:109AE00009F496C0833009F457C0813041F00895DD
:109AF0008A3009F480C08B3009F468C008958091E1
:109B0000D50D813A09F047C08091E800877F8093A6
:109B1000E8008091D90D9091DA0D892B59F060E021
:109B200080E090E070E033D28091E8008B77809302
:109B3000E800089568E08FEE99E0F4CF8091D50DAC
:109B4000813249F58091D90D9091DA0D8D7F892B65
:109B500011F58091E800877F8093E8008091E8000C
:109B600082FF15C08091F2009091F300029731F4CA
:109B70008091F100813011F0863019F48091F1006C
:109B800006DC8091E8008B778093E800E9C2809141
:109B9000D40D8111E3CF08958091D50D813AD9F785
:109BA0008091D90D9091DA0D892BA9F78091E80069
:109BB000877F8093E8008091E80080FFFCCFE4DBA2
:109BC0008093F1008091E8008E77DECF8091D50DF3
:109BD000813209F78091D90D9091DA0D892BD9F650
:109BE0008091E800877F8093E800BAD28091D70DFA
:109BF000BCDB0C9415138091D50D813261F68091F8
:109C0000E800877F8093E800ABD28091D80DCDCB60
:109C10008091D50D813A09F0BECF8091E800877F11
:109C20008093E8008091E80080FFFCCFC9DBC8CFBB
:109C30009FB7F8941092EE099FBF9091D40D943085
:109C400009F047C02091E9009091EC002F709795A2
:109C500099279795922B25E02093E9002091EB001E
:109C600020FF34C02091EE0027FF30C02091EC0986
:109C7000211521F02091E80025FF28C01092EC0961
:109C800026E03091E80035FF14C08093F100809108
:109C9000E80085FD27C08091E80080FFFCCF80911F
:109CA000E8008E778093E8009F709093E90080E051
:109CB00008953091D40D343049F43091EB0035FDE6
:109CC00005C02A9541F481E08093EC099F70909340
:109CD000E9008FEF0895EFE9FFE03197F1F700C059
:109CE0000000CFCF8FB7F89421E02093EE098FBF0B
:109CF000DBCF84B7877F84BF0FB6F894A895809197
:109D00006000886180936000109260000FBE80E860
:109D100090E00FB6F89480936100909361000FBEBD
:109D200022CB6ED2CAD2E2EEF0E0808184608083E2
:109D3000789438C584E391E01DC98091D40D8530B5
:109D400029F48091D40D853011F0BCCB08958FDBC0
:109D500042DB8115B1F38091D20D811591F367D06B
:109D60000E941513EECF08959A014091DB0D50919A
:109D7000DC0D00C0AC01CB01D901252F33272330E6
:109D80003105D1F070F42130310509F44BC0223097
:109D9000310569F484E790E02FED35E12D933C9394
:109DA00008952132310509F12232310559F180E05F
:109DB00090E020E030E0F2CFCA019927423091F0E4
:109DC0008330910538F4E9EBF5E1892B39F4EBEDBB
:109DD000F5E104C0EDE8F5E1039749F7849190E0DF
:109DE0009F01DCCFEBEAF5E1F9CF84309105F8F67D
:109DF000FC01EE0FFF1FEA5BFC4F2081318189E0FF
:109E000090E0CCCF8430910590F6FC01EE0FFF1F5F
:109E1000E25CFC4F20813181865C9C4FFC0180819B
:109E200090E0BCCF82E190E023E536E1B7CF84E15A
:109E300089BD86E189BD09B400FEFDCF8091D800BF
:109E40008F7D8093D8008091E00082608093E00055
:109E50008091E00081FDFCCF0895AF92BF92CF9238
:109E6000DF92FF920F931F93CF93DF936C01EB016F
:109E70008A0195D1F82E811123C00115110539F001
:109E8000F80180819181C81BD90BC80ED91EA12C65
:109E9000B12C2097A9F08091E80085FD21C0809128
:109EA000E8008E778093E80001151105A1F0F80114
:109EB000808191818A0D9B1D9183808385E0F82E9E
:109EC0008F2DDF91CF911F910F91FF90DF90CF9059
:109ED000BF90AF90089563D18115E9F2F82EF0CFCD
:109EE000F60181916F018093F1002197FFEFAF1A86
:109EF000BF0ACFCFAF92BF92CF92DF92FF920F9364
:109F00001F93CF93DF936C01EB018A0148D1F82EA8
:109F1000811123C00115110539F0F801808191816B
:109F2000C81BD90BC80ED91EA12CB12C2097A9F0A3
:109F30008091E80085FD21C08091E8008B778093B7
:109F4000E80001151105A1F0F801808191818A0DC9
:109F50009B1D9183808385E0F82E8F2DDF91CF911B
:109F60001F910F91FF90DF90CF90BF90AF90089519
:109F700016D18115E9F2F82EF0CF8091F100F601AB
:109F800081936F012197FFEFAF1ABF0ACFCFFC017A
:109F90009B018091DB0D9091DC0D8617970718F0DF
:109FA000672B61F0C90140E0009771F441110CC0CA
:109FB0008091E80082FF35C080E008958091E8003C
:109FC0008E778093E800EECF2091D40D2115A9F172
:109FD0002530A9F12091E80023FD2DC02091E80053
:109FE00022FDE6CF2091E80020FFDECF2091F20095
:109FF0003091F300009719F02830310558F041E016
:10A000002830310509F040E02091E8002E772093B8
:10A01000E800CACF41914093F10001972F5F3F4F75
:10A02000E9CF8091D40D811541F0853041F08091C8
:10A03000E80083FFBDCF81E0089582E0089583E0CA
:10A040000895FC019B018091DB0D9091DC0D86173A
:10A05000970718F0672B61F0C90140E0009771F491
:10A0600041110CC08091E80082FF36C080E0089565
:10A070008091E8008E778093E800EECF2091D40D98
:10A080002115B1F12530B1F12091E80023FD2EC05A
:10A090002091E80022FDE6CF2091E80020FFDECFEE
:10A0A0002091F2003091F300009719F0283031052B
:10A0B00058F041E02830310509F040E02091E800F7
:10A0C0002E772093E800CACF44914093F100319657
:10A0D00001972F5F3F4FE8CF8091D40D811541F05C
:10A0E000853041F08091E80083FFBCCF81E0089586
:10A0F00082E0089583E00895982F973028F08F70BC
:10A100008093E90081E008959093E900242F762F51
:10A1100050E0981731F07091EC002091ED005091D3
:10A12000F00021FD02C09F5FE8CF3091EB003E7F41
:10A130003093EB003091ED003D7F3093ED00309196
:10A14000EB0031603093EB007093EC002093ED0056
:10A150005093F0002091EE0027FDE5CF80E00895B8
:10A160008091D50D87FF13C08091E80082FF06C063
:10A170008091E8008B778093E80008958091D40D5A
:10A180008111F2CF08958091D40D8115D9F380917A
:10A19000E80080FFF8CF8091E8008E77ECCF209127
:10A1A000E4003091E50095E6A9012091EC00822FB2
:10A1B000817020FF06C08091E80080FF06C080E02B
:10A1C00008952091E80022FD1AC08091D40D8115D8
:10A1D00089F0853089F08091EB0085FD0FC02091DA
:10A1E000E4003091E50042175307F9F29A95E1F641
:10A1F00084E0089582E0089583E0089581E0089561
:10A200006AD071D0E0EEF0E0808181608083E8ED7B
:10A21000F0E080818F77808319BCA7EDB0E08C914E
:10A220008E7F8C9380818F7E80831092D30D0895D2
:10A230000F931F93CF93DF934ED055D0C8EDD0E04E
:10A2400088818F77888388818068888388818F7DE3
:10A250008883E7EDF0E080818068808319BC1092EC
:10A26000D40D1092D00D1092D20D1092D10D00EE9F
:10A2700010E0F80180818B7F8083888181608883F2
:10A2800042E060E080E038DFE1EEF0E080818E7F48
:10A290008083E2EEF0E0808181608083808188604D
:10A2A0008083F80180818E7F8083888180618883AC
:10A2B000DF91CF911F910F910895E8EDF0E080813B
:10A2C0008F7E8083E7EDF0E080818160808381E094
:10A2D0008093D30DADCFE8EDF0E080818C7F80835B
:10A2E0001092E20008951092DA001092E1000895B1
:10A2F0001F920F920FB60F9211240BB60F922F934D
:10A300003F934F935F936F937F938F939F93AF93FD
:10A31000BF93EF93FF938091E10082FF0AC0809189
:10A32000E20082FF06C08091E1008B7F8093E10014
:10A3300075DB8091DA0080FF18C08091D80080FF23
:10A3400014C08091DA008E7F8093DA008091D9006A
:10A3500080FF91C084E189BD86E189BD09B400FE1A
:10A36000FDCF81E08093D40D0CDB8091E10080FF74
:10A3700018C08091E20080FF14C08091E2008E7FBF
:10A380008093E2008091E20080618093E2008091FE
:10A39000D80080628093D80019BC85E08093D40DEA
:10A3A0001BDB8091E10084FF28C08091E20084FFE4
:10A3B00024C084E189BD86E189BD09B400FEFDCFDA
:10A3C0008091D8008F7D8093D8008091E1008F7EAE
:10A3D0008093E1008091E2008F7E8093E200809183
:10A3E000E20081608093E2008091D00D811509F434
:10A3F00047C084E08093D40DFFDA8091E10083FFB1
:10A4000027C08091E20083FF23C08091E100877F15
:10A410008093E10082E08093D40D1092D00D809162
:10A42000E1008E7F8093E1008091E2008E7F809337
:10A43000E2008091E20080618093E20042E060E00F
:10A4400080E05ADE8091F00088608093F000B8DAF6
:10A45000FF91EF91BF91AF919F918F917F916F91FC
:10A460005F914F913F912F910F900BBE0F900FBEB8
:10A470000F901F90189519BC1092D40D96DA75CFD5
:10A480008091E30087FF02C083E0B4CF81E0B2CFC8
:10A490001F920F920FB60F9211240BB60F92EF92EC
:10A4A000FF920F931F932F933F934F935F936F935D
:10A4B0007F938F939F93AF93BF93CF93EF93FF932C
:10A4C00009EE10E0F8018081C091EC008F70C79513
:10A4D000CC27C795C82B108280EFE82EF12CF7010E
:10A4E0008081877F8083789421D0F8011082F701E2
:10A4F000808188608083CF70F801C083FF91EF91E5
:10A50000CF91BF91AF919F918F917F916F915F910B
:10A510004F913F912F911F910F91FF90EF900F90CE
:10A520000BBE0F900FBE0F901F901895AAE2B0E0DF
:10A53000EBE9F2E515C285ED9DE0FC010196209165
:10A54000F10020832DE08D3D9207B9F7C3DA8091A9
:10A55000E80083FF37C08091D50D9091D60D9A30D9
:10A5600088F5E92FF0E0ED51F94AA6C1803889F06D
:10A57000823841F58091D90D8F70873018F580931E
:10A58000E9008091EB0085FB882780F91092E900B3
:10A5900006C08091D20D880F9091D10D892B90919A
:10A5A000E800977F9093E8008093F1001092F1000B
:10A5B0008091E8008E7722C0811115C08091D70D5F
:10A5C000813001F18091E80083FF0AC08091E800AA
:10A5D000877F8093E8008091EB0080628093EB009E
:10A5E000AA96E3E0D9C1823069F78091D70D811531
:10A5F00081F01092E9008091E800877F8093E80065
:10A60000AFDDE0CF81E0933009F080E08093D20DA0
:10A61000F0CF8091D90D8F702FEF280F263090F654
:10A620008093E9002091EB0020FFE3CF933031F4D9
:10A630008091EB0080628093EB00DBCF9091EB0088
:10A6400090619093EB0021E030E0A90102C0440F3B
:10A65000551F8A95E2F74093EA001092EA00809134
:10A66000EB008860E8CF8111ADCF1091D70D1F7737
:10A670008091E3008078812B8093E3008091E80053
:10A68000877F8093E8006CDD8091E80080FFFCCF3D
:10A690008091E30080688093E30083E0111101C0A2
:10A6A00082E08093D40D8ECF8058823008F08ACF1C
:10A6B0008091D70D9091D80D8C3D53E0950791F581
:10A6C00083E08A838AE289834FB7F894DE01139688
:10A6D00020E03EE051E2E32FF0E0509357008491F8
:10A6E00020FF03C082958F703F5F8F708A30C0F06B
:10A6F000895C90E08D939D932F5F243161F74FBF6C
:10A700008091E800877F8093E8006AE270E0CE01E4
:10A7100001963DDC8091E8008B778093E80052CF72
:10A72000805DE7CF6091D90D7091DA0DAE014F5F7A
:10A730005F4F1ADBBC01892B09F444CF8091E800FC
:10A74000877F8093E80089819A817BDCE3CF803822
:10A7500009F038CF8091E800877F8093E8008091EE
:10A76000D00D8093F10024CF81112CCF9091D70D83
:10A77000923008F027CF8091E800877F8093E8002F
:10A780009093D00DEDDC8091D00D811529F084E0FF
:10A790008093D40D82D916CF8091E30087FDF7CF47
:10A7A00081E0F6CFCF938091D40D811591F0809107
:10A7B000E900C091EC008F70C795CC27C795C82BD6
:10A7C0001092E9008091E80083FDB0DECF70C09365
:10A7D000E900CF910895DB018F939F93A8D0BF919B
:10A7E000AF91A29F800D911DA39F900DB29F900DE0
:10A7F00011240895992778E0880F991F961708F07B
:10A80000961B881F7A95C9F78095089587FB082EB7
:10A81000062687FD819567FD6195ECDF0EF4919525
:10A8200007FC81950895AA1BBB1B51E107C0AA1F15
:10A83000BB1FA617B70710F0A61BB70B881F991FE1
:10A840005A95A9F780959095BC01CD01089597FB85
:10A85000072E16F4009406D077FD08D0E4DF07FC3D
:10A8600005D03EF4909581959F4F08957095619520
:10A870007F4F0895A1E21A2EAA1BBB1BFD010DC03C
:10A88000AA1FBB1FEE1FFF1FA217B307E407F507A0
:10A8900020F0A21BB30BE40BF50B661F771F881F7C
:10A8A000991F1A9469F760957095809590959B0112
:10A8B000AC01BD01CF010895EE0FFF1F0024001C65
:10A8C0000BBE0790F691E02D0994082E8170069436
:10A8D0000694811D0694811D0694811D0694811D98
:10A8E0000694811D0694801D08956927962769277F
:10A8F000782787277827089505D0332312F48A1BF9
:10A900009B0B10C0A29FB001B39FC001A39F700D0D
:10A91000811D1124911DB29F700D811D1124911D67
:10A920000895F0DFB7FF0895821B930B0895EADFC7
:10A93000A59F900DB49F900DA49F800D911D112493
:10A9400008952F923F924F925F926F927F928F92D3
:10A950009F92AF92BF92CF92DF92EF92FF920F93AE
:10A960001F93CF93DF93CDB7DEB7CA1BDB0B0FB6B8
:10A97000F894DEBF0FBECDBF09942A883988488875
:10A980005F846E847D848C849B84AA84B984C8840B
:10A99000DF80EE80FD800C811B81AA81B981CE0F02
:10A9A000D11D0FB6F894DEBF0FBECDBFED010895E7
:10A9B000002E083090F0982F872F762F652F542F78
:10A9C000432F322F22270850F4CF220F331F441F6A
:10A9D000551F661F771F881F991F0A95B2F7002D14
:10A9E000089597FD1094002E083098F00850232FFA
:10A9F000342F452F562F672F782F892F912DF4CF85
:10AA000015949795879577956795579547953795B9
:10AA100027950A95AAF71124002D08958F929F92E9
:10AA2000AF92BF92CF92DF92EF92FF92CF93DF93DC
:10AA3000EC01688179818A819B81611571058105AD
:10AA4000910521F464E279ED8BE597E02DE133EF98
:10AA500041E050E0D1D049015A019B01AC01A7EA85
:10AA6000B1E465DF6B017C01ACEEB4EFA5019401AC
:10AA7000E1D0DC01CB018C0D9D1DAE1DBF1DB7FFCC
:10AA800003C00197A109B04888839983AA83BB8337
:10AA90009F77DF91CF91FF90EF90DF90CF90BF90A5
:10AAA000AF909F908F900895B9CF80E091E0B6CF9E
:10AAB000A0E0B0E08093000190930101A093020117
:10AAC000B09303010895FB01DC0102C005900D92D3
:10AAD00041505040D8F70895FC014150504030F0AB
:10AAE00001900616D1F73197CF010895882799274D
:10AAF0000895FB01DC0104C08D910190801921F4BF
:10AB000041505040C8F7881B990B0895FB01DC01A8
:10AB100002C001900D9241505040D8F70895DC01D9
:10AB200001C06D9341505040E0F70895DC01CB0126
:10AB3000FC01F999FECF06C0F2BDE1BDF89A31964D
:10AB400000B40D9241505040B8F70895F999FECFE6
:10AB500092BD81BDF89A992780B50895A6E1B0E02D
:10AB600044E050E0E5CFA8E1B0E042E050E0E0CFC3
:10AB7000DC01A40FB51F4150504040F0CB01840FC1
:10AB8000951F2E9105D041505040D8F70895262F9B
:10AB9000F999FECF92BD81BDF89A019700B40216D3
:10ABA00039F01FBA20BD0FB6F894FA9AF99A0FBE81
:10ABB00008950396272FECDFEADF252FE9DF242F06
:10ABC000E7CF0196272FE4DFE2CFDC01CB0102C003
:10ABD0002D9105D041505040D8F70895262FF9996E
:10ABE000FECF1FBA92BD81BD20BD0FB6F894FA9A70
:10ABF000F99A0FBE01960895052E97FB16F400945E
:10AC00000FD057FD05D036DE07FC02D046F408C051
:10AC100050954095309521953F4F4F4F5F4F089588
:10AC200090958095709561957F4F8F4F9F4F0895B8
:10AC3000B7FF7DCE7CDE821B930B0895F894FFCF87
:10AC4000271127115E115E11CA11E7114F114F1123
:10AC5000EB11531260126012611F641F681F6C1F9A
:10AC6000701F741F781F7C1F801F841F881FD826A9
:10AC7000DC26E226DE26E026E426E62648296829A8
:10AC8000742964296429A629C429D729212A262AB6
:10AC90006429642964292D2A382A472A5E2A872AAA
:10ACA000972A64296429B12AC12A4E3735375F377C
:10ACB0008636F937F9372E37F937F9378F37F937BD
:10ACC0009F37E037F937F937F937F937BA37F937B6
:10ACD000F937AF37F9377837F937F937F737F737C3
:10ACE000F737F737F737F737F737F737F737F237F9
:10ACF000F9374E372337F937F937F937F937F93755
:10AD0000F937F937F937F937F937F237F937F937CA
:10AD10002E37F937F537F537F537F537F537F53796
:10AD2000F537F537F537F237AB3D1A3EB33D7D3D8C
:10AD3000813DB73D853DBB3DC73D913D133E953DB2
:10AD4000CB3D993DCF3DF43D9D3DD33DFB3DA33DE6
:10AD5000D93DE13D893DBF3D8D3DC33DA73DDD3D35
:10AD6000EB3D043E113E773DAF3D213EC03EC53E2A
:10AD7000C73ECC3EDC3EDC3EDC3EDC3EDC3EDC3E28
:10AD8000DC3EDC3ECE3ED23ED53EDA3EEA3EF03EF2
:10AD9000F43E6044664451445A446C4472447844DE
:10ADA000DD46E946144720472B47364739473E479B
:10ADB0004347D946A54748474C47544765477D47D1
:10ADC000804783479447B652DC52E252DC52E2524B
:0AADD00033535453E252A753B45317
:10ADDA0001000000FE031E04010102001E001E1EE7
:10ADEA0001191A1B1C1D1E1F202122060100210009
:10ADFA007F22000301280850011E0A1401030201E0
:10AE0A0000000100D2497C4C774C724C6D4C644C6A
:10AE1A00E200E900EA00B500B600B700CD00830100
:10AE2A00CC008A0192019401210223022402250204
:10AE3A00260227022A02B300B4006F0070009F01A5
:10AE4A00CB019F02A002E200E900EA00B500B600C9
:10AE5A00B700CD008301CC008A019201940121023E
:10AE6A00230224022502260227022A02B300B40082
:10AE7A006F0070009F01CB019F02A0020001020334
:10AE8A00040506076766656463626160F5F6F7F2B2
:10AE9A00F1F0C1C000010202020206060609090910
:10AEAA000909090F0F0F0F0F0F1515151819191981
:10AEBA00191919191919192324252525252525FBB9
:10AECA002FFD2F0830203015AA2F63C4EF61A3008D
:10AEDA003F3F3F006D6B5F64656C6179006D6B5F2E
:10AEEA00696E74657276616C006D6B5F6D61785F17
:10AEFA007370656564006D6B5F74696D655F746F0F
:10AF0A005F6D6178006D6B5F776865656C5F6D6119
:10AF1A00785F7370656564006D6B5F776865656CF3
:10AF2A005F74696D655F746F5F6D6178000A092DE2
:10AF3A002056657273696F6E202D0A5649443A206D
:10AF4A003078353434422822546865204B6579209C
:10AF5A00436F6D70616E792229205049443A20303E
:10AF6A00783030303428224D306C6C7922292056C2
:10AF7A0045523A203078303030310A4255494C44F3
:10AF8A003A2020284D617920313820323032362952
:10AF9A000A4F5054494F4E533A204C55464120428D
:10AFAA004F4F544D41474943204D4F5553454B450B
:10AFBA00592045585452414B455920434F4E534FFF
:10AFCA004C4520434F4D4D414E44204E4B524F204D
:10AFDA00383139320A4743433A2031342E322E303F
:10AFEA00204156522D4C4942433A20322E322E31BC
:10AFFA00204156525F415243483A206176723531B8
:10B00A000A0000081018181008004422B615521732
:0EB01A007A169C166516F1150A162A164316AC
:00000001FF
